:1000000087C30000BDC30000BBC30000B9C300002C
:10001000B7C30000B5C30000B3C30000B1C3000004
:10002000AFC30000ADC300000C940D320C94F53248
:100030000C94C231A5C30000A3C30000A1C30000FB
:100040009FC300009DC300009BC3000099C3000034
:1000500097C300000C94E93193C3000091C30000E2
:100060008FC300008DC300008BC3000089C3000054
:1000700087C3000085C3000083C3000081C3000064
:100080007FC300007DC300007BC3000079C3000074
:1000900077C3000075C3000073C3000071C3000084
:1000A0006FC300006DC300006BC300000501098031
:1000B000A101850319012AB700150126B700950192
:1000C00075108100C0050C0901A101850419012AE0
:1000D000A002150126A002950175108100C005013E
:1000E0000906A1018506050719E029E71500250184
:1000F0009508750181020507190029EF15002501F2
:1001000095F075018102050819012905950575010C
:100110009102950175039101C00660FF0961A1017B
:100120000962150026FF00952075088102096315F4
:100130000026FF00952075089102C005010906A15F
:1001400001050719E029E7150025019508750181CA
:10015000029501750881010507190029FF15002680
:10016000FF0095067508810005081901290515008D
:100170002501950575019102950175039101C00056
:10018000000000000000000000000000000000006F
:10019000000000000000000000000000000000005F
:1001A0000000007E0F00D4FFFFFFC70000007800B2
:1001B000000000000000002A2B28000000000000C2
:1001C0000000000000000000000029000000002CDA
:1001D0001E3420212224342627252E362D37382779
:1001E0001E1F202122232425263333362E37381F85
:1001F0000405060708090A0B0C0D0E0F1011121347
:100200001415161718191A1B1C1D2F3130232D35E4
:100210000405060708090A0B0C0D0E0F1011121326
:100220001415161718191A1B1C1D2F3130354C09BF
:10023000025B00030100A0FA0904000001030101B0
:100240000009211101000122440007058103080073
:10025000010904010002030000000921110100014D
:100260002222000705820320000107050303200066
:10027000010904020001030000000921110100012D
:10028000226D000705840320000112010002000016
:10029000000869EB03600100010203011C03760002
:1002A000690061006C003A006600360034006300AB
:1002B000320062003300630000000E034400690056
:1002C000610062006C006F0000000E036B006500AF
:1002D0007900740065006E00000004030904290021
:1002E0001E001F0020002100220023002400250002
:1002F000260027002D002E0035002B0014001A00C8
:100300000800150017001C0018000C001200130054
:100310002F003000310039000400160007000900EA
:100320000A000B000D000E000F00330034002800FF
:100330002A00E1001D001B00060019000500110045
:100340001000360037003800000000002152E000A5
:10035000E300E2000000000000002C0000000000AC
:100360000000E600E700E500E40001003A003B0081
:100370003C003D003E003F00400041004200430081
:1003800044004500010001000100010001000100DE
:100390000100010001000100010001000100010055
:1003A0000100010001000100010001000100010045
:1003B0000100010001000100010001000100010035
:1003C0000100010001000100010001000100010025
:1003D0000100010000000000010001000100010017
:1003E000000000000000010000000000000001000B
:1003F00001000100010001000100B10402165616BF
:10040000000002000200AD040216561600000300B0
:100410000100B20402165616000004000200970400
:1004200002165616F60705000100B304021656160A
:10043000000006000200990402165616000007008C
:100440000200AF0402165616000012000200B504A6
:1004500002165616000013000200B70402165616C4
:10046000000014000100B904021656160000150021
:1004700000000000FF079F0E000016000100B404FA
:1004800019166D16000017000101B40419166D1637
:10049000000018000102B40419166D1600001900BE
:1004A0000200BB040216561600001A000103B40431
:1004B00019166D1600001B000200BD040216561628
:1004C0000000FD377A585A000004E6D6B446020010
:1004D000210116000000742FE5A3E004EB01A05DEC
:1004E000003D8889C65436C3174FE4DD5EF0CFB6B1
:1004F000AAC3B64CAFD49697AC35E6F579BD503B60
:1005000024634C6222D1D52A359EBBF92EAB23FC45
:10051000146B346BDD70BD4B0D0A9927F3B4464262
:100520001990622F16AEE20529158D2C346A776872
:10053000A9EAC7E67280A899375A4B57C07DF8C51B
:10054000BE0CF0DF22B624E85648D4C8D3F5CE3C22
:10055000844A5544D2486B981AFE5E25420E04F533
:100560002C77E343E571F2001523C3A79259846603
:1005700085B0E0B44B7070CB709A06F0475BA8CEA4
:100580006FB936A412A5E2DB51AD7E5606ADC409A3
:10059000F3BE8A49D2B0ED1D45570309E920F53F66
:1005A0008CEC1B6EDD59635590A5BCF5298204E8DF
:1005B0004263630CE7481814A0C050F68ECB145663
:1005C00099C508E932BD8C5291CDABB8D674E124FF
:1005D000E61DDC6F26C22D1D9864B531E6E4C562C8
:1005E000AC012987261C00FB549A4B579B5DEDC13B
:1005F0007A7E5E1C07208179329C737340C41D058E
:10060000F9B47C3F645ADBE26895E42222B9626A5D
:10061000C5F7C3C0A6E5D5A25A226858947E2D6AB4
:10062000AC77992E558B7C30D33DD5E514E8548AB0
:10063000F97B2F2FA7EC3D995FE2EFE15C328D78DB
:100640005D2A9A8571F4492C0643562193F89078D7
:1006500034C15E2DCD84DA00C26B9B66FDBA7BCBC4
:1006600060DAA319B4F86831CFCD025AC014C57747
:100670002ACCCB8BBB205481DCE7FDA923D84A3D93
:100680000000BBA20EB45301240F0001BC03EC090F
:1006900000000CB8857AB1C467FB020000000004BA
:1006A000595A4C4C4C4C4C4C4C5252525252525245
:1006B0004C4C4C4C4C4C4C525252525252524C4C50
:1006C0004C4C4C4C4C525252525252524C4C4C4C40
:1006D0004C4C4C525252520000524C4C4C000000B8
:1006E0002A00000052525252504F52514A4D4B4E26
:1006F0002A4C2F30B6B7ABACBBBCA9AABDBE0D0E01
:100700000B0F1A0508050905071811130408120C28
:1007100011241FBECFEFDAE0DEBFCDBF04B603FE6B
:1007200018C08091C4049091C504A091C604B091F2
:10073000C7048730904BA740B04B59F41092C404C3
:100740001092C5041092C6041092C704E0E0F8E3CA
:10075000099511E0A0E0B1E0E0EBF8E602C00590F9
:100760000D92AC3AB107D9F724E0ACEAB1E001C090
:100770001D92A43CB207E1F70E94322B0C941B346B
:100780003FCC9C019A9581159F4118F5F32FF2708B
:10079000EE27832F8170732F74706627532F587044
:1007A000442734FF0CC08295807FEF2B09F08062D4
:1007B000672B09F08064452B69F080680895EF2B62
:1007C00009F08260672B09F08460452B19F088607E
:1007D000089580E00895CF93DF93EB01D2DFFE010F
:1007E0000995DF91CF9108950C9446330895982F81
:1007F00092959F7024E0911102C020E0982F892FDC
:1008000086958695811511F02E5F982F892F8695F4
:10081000820F0895282F92959F70963099F060F47A
:10082000925F9F70923030F4203FB1F038F481E055
:10083000283E38F080E008959A5FF3CF81E0243FAE
:10084000C9F7089591E0813F09F090E081E0283EEA
:1008500008F080E0892B089581E0089580933904A1
:10086000089580933A04089521E030E001C0220FFA
:100870008A95EAF780913A04822BF3CF21E030E0A9
:10088000A90102C0440F551F8A95E2F7CA0180955D
:1008900090913A048923E5CF292F953090F58E3039
:1008A00080F590E03EE0239F800D911D1124282FBC
:1008B000277041E001C0440F2A95EAF723E096959E
:1008C00087952A95E1F7FC01EE0FFF1FE80FF91F4E
:1008D000EF56FD4F20E030E070E05191DF01CB0199
:1008E000022E02C0969587950A94E2F78170819551
:1008F0008527842385278E932F5F3F4F2330310533
:1009000061F70895292F953078F58E3068F590E0DD
:100910003EE0239F800D911D1124682F677023E016
:10092000969587952A95E1F7FC01EE0FFF1FE80FDA
:10093000F91FEF56FD4F40E050E080E0219130E09C
:10094000062E02C0369527950A94E2F721703327C8
:10095000042E01C0220F0A94EAF7822B4F5F5F4FEB
:100960004330510559F7089580E0089590913A0475
:1009700021E030E0F90101C0EE0F8A95EAF7D901D4
:1009800002C0AA0FBB1F6A95E2F7EA2B01C0220F33
:100990004A95EAF7892F8E23E81303C0892F822B0B
:1009A00060CF2095822F8923FBCF8091900290E029
:1009B00020E0022E001C0008281709060CF00895FC
:1009C0002F5FF7CFFC01DB018481813041F5149664
:1009D0008C911497813019F591818EE0E081F0E0DF
:1009E000899FE00DF11D1124EE55F94F94919A3233
:1009F000B1F011962C911197EC91F0E0829FE00DEF
:100A0000F11D1124EE55F94FE49181E09E1301C0D0
:100A100080E091E0EA3209F090E0892B089581E0CE
:100A200008959C0180913B048D79811119C0211595
:100A300040E5340780F4211580E23807C0F4233301
:100A4000310511F1D0F481E02E31310590F42430DC
:100A5000310530F00895C90196558115914010F087
:100A600080E00895C901805F96450797C8F3332752
:100A7000E6CF2C323105A1F708952653310981E0E4
:100A80002330310538F3ECCF81E00895809145049F
:100A900090914404981301C008958F5F8770FACF36
:100AA00090913F048095892380933F04282F2770DD
:100AB000211110C0891771F09091C00492FF0AC0F3
:100AC000869586958695DADE10923F041092410451
:100AD00010924004089590913B04982B90933B040E
:100AE0000895982F909580913B04892380933B042F
:100AF0000895982F909580913E04892380933E0419
:100B0000089580913704811531F0109237041092C6
:100B10003604109235040895803E9105D9F1C8F449
:100B20008133910509F482C048F48932910509F4B2
:100B300072C08A32910509F480C008958933910505
:100B4000E9F082389105D1F08533910509F45EC052
:100B50000895843E9105D9F148F4823E910539F11A
:100B6000833E910549F181EE90E00895863E91051E
:100B7000C9F1873E910509F43EC008952091BF0454
:100B80002370211164C02091C00423FF14C089E2A6
:100B900090E008952091BF0420FD45C03091C0042D
:100BA00030FF09C024FD24C083EE90E00895209119
:100BB000BF0422FDF7CF08952091BF0422FD44C059
:100BC0003091C00430FD43C024FFF5CF11C0209107
:100BD000C00421FFF0CF8091BF0484FD09C087EEDF
:100BE00090E008952091BF0423FFE5CF24FFF7CFC5
:100BF00080E090E008952091BF0423FD2BC0309148
:100C0000C00431FFE1CF84EE90E008952091BF044D
:100C100025FFD1CFBCCF2091BF0425FD1EC0209160
:100C2000C00423FFC8CF89E390E008952091BF045A
:100C300026FFC1CF8AE290E008952091BF0426FFED
:100C4000BACF81E390E0089582EE90E0089580EEBF
:100C500090E0089586EE90E0089585E390E0089591
:100C60009091BF0492FF10C041E0282F24712430DE
:100C700009F040E031E0282F2871283009F030E0F9
:100C8000431711F02CE0822793FF10C041E0282F7A
:100C90002471243109F040E031E0282F28712831F7
:100CA00009F030E0431711F02CE082273091C004A6
:100CB00030FF10C051E0282F2171213009F050E0A1
:100CC00041E0282F2871283009F040E0541711F036
:100CD00029E0822731FF10C041E0282F2171213106
:100CE00009F040E031E0282F2871283109F030E088
:100CF000431711F029E0822794FD877E08951F9302
:100D0000CF93DF9309DFEC01811522E5920708F00C
:100D100052C0811540E5940708F0CDC0803E910592
:100D200020F58D3C910508F0A1C0883A910570F43A
:100D3000853A910508F097C081309105B9F1049783
:100D4000813A910598F1C0E0D0E030C0885A91090D
:100D50004B97C8F7C85AD0E0CC0FDD1FC05CDE4F00
:100D60000990D881C02DD46421C0811550E4950725
:100D7000B0F4C11580E2D80708F0B3C0C83ED10571
:100D8000A8F0CE019A9581159F41E8F68D2F68DF76
:100D9000182FCE019927C0DEEC01D12B07C099276F
:100DA000BBDECC27DF70C82BD92BD06ACE01DF91F8
:100DB000CF911F910895803842E59407C8F5803699
:100DC00052E5950708F05BC0C03482E5D807D0F43F
:100DD000C03292E5D90708F04BC08C2F86958695D6
:100DE00020E2829FC0011124C37021E030E0A901FC
:100DF00002C0440F551FCA95E2F7EA01C82BD92B50
:100E0000DD68D4CF8C2F86958695877050E2859FBC
:100E1000C0011124C37021E030E0A90102C0440FD9
:100E2000551FCA95E2F7EA01C82BD92BDC68BECF63
:100E3000803C52E5950758F48F71C03AD245A0F531
:100E400090E0982F8827EC01C46FD06AAFCF805C08
:100E50009245809708F077CFDC2FCC27CC27DF7125
:100E6000C06FD06AA3CFA497D064A0CFD0659ECF27
:100E7000CF71D0E0DC2FCC27C16FD06A97CF869599
:100E80008695877020E2829FC0011124C37021E003
:100E900030E0A90102C0440F551FCA95E2F7EA01EC
:100EA000C82BD92BDA6882CFDBDEC82FD0E0DC2F4D
:100EB000CC27D0627BCF8F71D3DE93E0CC0FDD1FC8
:100EC0009A95E1F7CC27DF70282F30E084FF05C02A
:100ED00050E1859F900111243327C22BD32BD06979
:100EE00065CF8D2F8F71BCDE182FCE01992714DEB0
:100EF000EC01D12BDECF80E00895F894E82FE29545
:100F0000EF70F0E041A18F7021E030E0B90102C044
:100F1000660F771F8A95E2F7CB01962F9095942361
:100F200091A392A1892B82A37894089581152CE72F
:100F3000920741F420914D0230914E02232B11F47F
:100F400080E090E00895E1EAF3E080E090E06AE478
:100F50007AE24DE65AE22FED3AE2778366835187D3
:100F600040873387228797878687019670968830D7
:100F7000910599F70895FB01811520E2920728F465
:100F8000811541E0940738F408959C0130522115F1
:100F9000304348F00895392F94FF02C03295307FD6
:100FA0002081232B208399270895462B22FF0FC0F1
:100FB000982F92959F708F70892B962F92959F7086
:100FC0006F70692B942F92959F704F70492B982FBB
:100FD0009623961309C050E04095509590E0482321
:100FE000592381E0452B09F080E008958091970412
:100FF0009091980490930D0180930C010895EF92C5
:10100000FF920F931F93CF93DF93FB018FEF9FEF1F
:101010004430510508F45FC04091BF0441FB88276C
:1010200080F990E0880F991F42FB002700F910E03B
:10103000000F111F000F111F802B912B40FBEE247E
:10104000E0F8F12C8E299F2943FB222720F9C22F9B
:1010500050E0D52F53E0CC0FDD1F5A95E1F78C2BD4
:101060009D2B44FB222720F950E1259F900111245C
:10107000822B932B45FB222720F950E2259F9001DC
:101080001124822B932B46FB222720F950E4259F25
:1010900090011124822B932B47FB222720F940E853
:1010A000249F90011124822B932B2091C004322F76
:1010B0003170932B26952170B22FBB0FA0E08A2BA5
:1010C0009B2B092E000CAA0BBB0B80839183A28360
:1010D000B38380E090E0CDB7DEB7E6E00C948533D3
:1010E000AC0123E0969587952A95E1F78E719927B3
:1010F000FC01EA50FE4F0190F081E02D4F70552722
:1011000021E030E002C0220F331F4A95E2F761155B
:1011100041F0E22BF32B8A509E4FDC01ED93FC93C0
:10112000089520953095E223F323F5CFFC018481C7
:10113000862381110AC082818115B9F068239085C8
:1011400093FF05C081E061110FC080E00895282F52
:1011500022952F708F70282B962F92959F706F700D
:10116000962B81E02913F1CF089581E008950F9324
:101170001F93CF9301E010E0082E01C0000F0A94E6
:10118000EAF7C09134049C2F9023911115C09091DF
:101190003F04969596959695891306C010923F0444
:1011A00010924104109240045FDBC027C0933404C6
:1011B000CF911F910F91089561DBF7CF90910303B9
:1011C00089029001112437FF03C08093030308951F
:1011D0002F3731051CF4980F9093030308959C0159
:1011E00080E090E0F901E80FF91FE491E41307C0F3
:1011F00091E08927F901E80FF11D84910895019686
:10120000861780F380E00895FA01309709F0099578
:101210000895E0917602F0917702309739F00190CD
:10122000F081E02D309711F00995089580E0089540
:10123000A3E0B0E0EEE1F9E00C946D339C01809105
:10124000F4019091F50182179307B1F03093F50105
:101250002093F401E0917602F0917702309761F0EB
:101260000084F185E02D309739F083E089833B835A
:101270002A83CE01019609952396E2E00C948933E6
:10128000A3E0B0E0E6E4F9E00C946D339C018091BA
:10129000F2019091F30182179307B1F03093F301BB
:1012A0002093F201E0917602F0917702309761F09D
:1012B0000084F185E02D309739F084E089833B8309
:1012C0002A83CE01019609952396E2E00C94893396
:1012D00090911001913091F0A0EBB1E0EFEF90E030
:1012E0002D91821751F0EF3F19F4211101C0E92F20
:1012F0009F5F9630A9F7EF3FC9F408959091BF041E
:1013000097FFEACFE82FE695E695E695803FA8F7A8
:10131000F0E0EA54FE4F877021E030E001C0220F78
:101320008A95EAF78281822B828308950E2E000C23
:10133000FF0BE255FE4FF8CF90911001913021F450
:101340009091BF0497FD0CC0E0EBF1E091918913FF
:1013500002C0DF011E9251E0E63BF507B9F70895A0
:10136000E82FE695E695E695803FC8F7F0E0EA5469
:10137000FE4F877021E030E0A90102C0440F551FE5
:101380008A95E2F7CA018095928189238283089524
:1013900080910F0108952FB7F8948091EE019091FC
:1013A000EF01A091F001B091F1012FBF089580915C
:1013B000990490919A04892B89F0EDDF20913504EE
:1013C00030913604AC01421B530B9A0181E04091ED
:1013D000990450919A042417350708F480E0089581
:1013E000CF93DF93C0913B0480913E04C82B809142
:1013F00037048115E1F08091990490919A04892B2A
:1014000019F0D5DF81117DDBD09137048091100177
:10141000813021F48091BF0487FD13C086E020EB6A
:1014200031E090E0815088F491116BDBCD2B8091FD
:101430001D0380958C2390911C03892BDF91CF9104
:1014400008958EE128EB31E0ECCFF90141919F0145
:10145000411541F39F5FE6CF962F2091C00422FFF4
:101460000EC0682F660F660F660F692B60933F04EE
:10147000FBD991DF90934104809340040895F4C90F
:1014800090913704292F2823211559F0809589231D
:1014900080933704811531F07EDF8093350490937B
:1014A0003604089580E090E0F8CFCF93C82F809164
:1014B000C00482FF0BC0809137048C1739F06BDFBA
:1014C0009093360480933504C0933704CF910895E8
:1014D0002FB7F8946091EE017091EF018091F001C7
:1014E0009091F1012FBF0895CF92DF92EF92FF927A
:1014F000CF93DF93D82FC92FC0909B03D0909C032C
:10150000E0909D03F0909E03E3DF6C197D098E0946
:101510009F09643F71408105910510F1D9DF6B018E
:101520007C0182E390E0A0E0B0E0C0923A02D09269
:101530003B02E0923C02F0923D028093360290938F
:101540003702A0933802B0933902D0939903C09325
:101550009A03DF91CF91FF90EF90DF90CF900895A5
:1015600084EF91E0A0E0B0E0E0CF0895FC019B01A2
:101570008091E4019091E5018617970740F0672B71
:1015800029F48091E8008E778093E800C90140E05B
:10159000009741F4411106C08091E80082FF2FC0FE
:1015A00080E0089520914F022115A9F12530A9F17D
:1015B0002091E80023FD2DC02091E80022FDECCF12
:1015C0002091E80020FFE4CF3091F3002091F20059
:1015D000009719F02830310558F041E028303105E6
:1015E00009F040E02091E8002E772093E800D0CF6A
:1015F00041914093F10001972F5F3F4FE9CF8091D8
:101600004F02811541F0853041F08091E80083FF61
:10161000C3CF81E0089582E0089583E0089580912A
:10162000DE0187FF13C08091E80082FF06C0809131
:10163000E8008B778093E800089580914F02811134
:10164000F2CF089580914F028115D9F38091E8007F
:1016500080FFF8CF8091E8008E77ECCF2091E400F6
:101660003091E50095E6A9012091EC00822F817070
:1016700020FF06C08091E80080FF06C080E008954A
:101680002091E80022FD1AC080914F02811589F057
:10169000853089F08091EB0085FD0FC02091E4003A
:1016A0003091E50042175307F9F29A95E1F684E08C
:1016B000089582E0089583E0089581E00895E8EDBB
:1016C000F0E080818E7F80831092E2001092DA0039
:1016D0001092E100A0EEB0E08C9181608C9380814B
:1016E0008F77808319BCA7EDB0E08C918E7F8C93AF
:1016F00080818F7E80831092DD010895E0917602D3
:10170000F0917702309739F00284F385E02D30971D
:1017100011F060E209950895982F9093E9008917D8
:1017200071F07091EC002091ED005091F00021FDDE
:1017300009C09F5F973089F78093E9000895762F5D
:10174000242F50E03091EB003E7F3093EB0030913E
:10175000ED003D7F3093ED003091EB003160309330
:10176000EB007093EC002093ED005093F00020917B
:10177000EE0027FDDECF0895A0E0B0E0E2ECFBE054
:101780000C946733C8EDD0E088818F7E8883E7EDC5
:10179000F0E080818160808384E082BF81E080937B
:1017A000DD0188818E7F888302EE10E0F8011082CF
:1017B0001092DA0081EEC82ED12CF60110828881B9
:1017C0008F77888388818068888388818F7D8883EC
:1017D00019BC10924F021092DC0110922A02109252
:1017E000DB0190EEE92EF12CF70180818B7F808365
:1017F00088818160888342E060E080E08DDFF601CF
:1018000080818E7F8083F8018081816080838081E8
:1018100088608083F70180818E7F808388818061EA
:101820008883CDB7DEB7E8E00C948333E0914504BC
:101830009091440429E0E91302C080E00895AE2F9E
:10184000B0E02E9FF0011124EA5BFB4F318136138B
:1018500006C03081381303C03581341304C0FD0144
:101860003196E770E8CF81E008959C01211531059C
:1018700009F408958FE99FE00197F1F700C0000097
:1018800021503109F3CF81E08093E00080E2809322
:10189000D8001092C9008FE19EE40197F1F700C0D3
:1018A000000087E090EBDC018093C4049093C504B2
:1018B000A093C604B093C70488E19CE00FB6F894E7
:1018C000A895809360000FBE90936000FFCF0F93A8
:1018D0001F93CF93DF938B01EA0190914F029430D5
:1018E00051F58093E9008FEF9091E80095FD06C0D7
:1018F00095ED9A95F1F700008A95B1F78091E8008F
:1019000085FF19C0ABDE811111C08091E80085FD13
:1019100006C08091E8008E778093E800F3CFF8014D
:1019200081918F018093F100219779F78091E800F0
:101930008E778093E800DF91CF911F910F910895EA
:10194000792F603229F440E250E0682F82E0BFCF67
:101950000895CF93DF93D82FC92F48E050E0682F28
:10196000792F81E0B4DF88E0ED2FFC2FA6EEB1E007
:1019700001900D928A95E1F7DF91CF910895BC0116
:1019800040E250E084E0A3CFBC0143E050E084E0BB
:101990009ECF9091C00492FB222720F9281771F066
:1019A00080FB92F99093C0046091BF047091C004D1
:1019B00084E090E00E94003482E072C808951F9392
:1019C000CF93DF93962F122F632F8430D8F4953066
:1019D000C8F44E30B8F4C42FD0E0CC0FDD1F2CE19A
:1019E000929FC00DD11D11249CE8899FC00DD11D6F
:1019F0001124CE0189960E94E633612FCE018A968A
:101A00000E94E633DF91CF911F91089580911001DC
:101A1000813061F58091BF0487FF28C0E1DC8093AD
:101A2000B70140E250E066E572E086EB91E00E948B
:101A30009D33892BD1F080E2E6EBF1E0A6E5B2E040
:101A400001900D928A95E1F7E0917602F09177028C
:101A5000309759F00480F581E02D309731F086E021
:101A60008093B60186EB91E009950895B9DC8093E7
:101A7000AE0148E050E068E772E08EEA91E00E9433
:101A80009D33892B91F388E0EEEAF1E0A8E7B2E01C
:101A900001900D928A95E1F7E0917602F09177023C
:101AA000309719F30280F381E02D3097F1F28EEA3E
:101AB00091E0DACF811511F00ED8A8CF08958115E5
:101AC00031F090913E04892B80933E049FCF08957E
:101AD000811511F006D89ACF0895811511F009D813
:101AE00095CF089580911803811521F082E2F5DFEA
:101AF000109218030895CF93C82F8115C1F08CEF71
:101B00008C0F813A80F580911001813021F4809111
:101B1000BF0487FD0EC0E0EBF1E08191C817F9F03A
:101B200021E0E63BF207C9F78C2FD2DB6FDFCF91C4
:101B30000895EC2FE695E695E695F0E0EA54FE4F21
:101B4000828190E04C2F477021E030E002C0220FEC
:101B5000331F4A95E2F782239323892B29F38C2F95
:101B6000EBDB54DFE1CF80E28C0F883048F4C770A4
:101B700081E001C0880FCA95EAF70E946B05D6CFB5
:101B80008BE58C0F833030F42C2F2452330BC9019A
:101B90004FDBCDCFC85ACB3150F6EC2FF0E0EE0F33
:101BA000FF1FEA58FE4F808191816ADBC0CFCF933F
:101BB000DF93EC01805E9109089720F06FE57DE0EE
:101BC000209711F46AE57DE0CE010E94EB038C2F93
:101BD00092DFDF91CF910895611529F020913E04A5
:101BE000226020933E049C0130522115304308F4BA
:101BF0009927DDCF811509F19CEF980F913A10F4E8
:101C00009BDB04CF90E2980F983050F4877091E0FE
:101C100001C0990F8A95EAF7892F0E947105F1CFCB
:101C20009BE5980F933018F480E090E001CB885A40
:101C30008B3118F480E090E023CB0895CF93DF93AD
:101C4000EC01D8DFCE01805E9109089720F06DE6A7
:101C50007DE0209711F468E67DE0CE010E94EB0361
:101C6000DF91CF9108951F93CF93DF93182FEB014E
:101C700042DF209731F4812FBDDFDF91CF911F919B
:101C800008958FE99FE00197F1F700C000002197C8
:101C9000F0CF6091B7047091B804893321F060915E
:101CA000B5047091B604DFCF10923B04809110010F
:101CB0008130A1F48091BF0487FF10C0E8EBF1E010
:101CC0008EE1DF011D928A95E9F780E090E0B0DABD
:101CD00080E090E0D5DA10923E0498CEE0EBF1E09F
:101CE00086E0EFCFE1DF2FEF84E39CE021508040DE
:101CF0009040E1F700C0000088E19CE00FB6F89446
:101D0000A895809360000FBE90936000FFCFCF93A3
:101D1000DF93D82FC92F20919002283010F0C4DF14
:101D200020E0E22FF0E0EE0FFF1FE058FD4FD083E0
:101D3000C1832F5F20939002DF91CF910895CF93BD
:101D4000DF93FB018FEF9FEF44305105B0F0D0815E
:101D5000C181AADFD093BF04C3708091C0048C7F7F
:101D6000C82BC093C0046091BF047091C00484E08C
:101D700090E00E94003480E090E0DF91CF910895E0
:101D8000AAE2B0E0E6ECFEE00C946C338EED91E05C
:101D9000FC0101962091F100208321E0863E92070C
:101DA000B9F78091DF01893009F457C0C8F4823057
:101DB00009F4B2C0833009F482C0813081F180918E
:101DC000E80083FFE6C08091DE019091DF019A3048
:101DD00008F0DFC0E92FF0E0E35EFB4C0C944033E9
:101DE0008A3009F489C08B3051F78091DE0181324D
:101DF00031F78091E2019091E301892B01F7809105
:101E0000E800877F8093E8000ADC81E09091E001A0
:101E1000911101C080E08093100146DFD0CF809106
:101E2000DE01813A61F68091E800877F8093E800C7
:101E30008091E2019091E301892B59F060E080E00C
:101E400090E070E093DB8091E8008B778093E8006E
:101E5000B6CF68E086EE91E0F4CF8091DE0181326A
:101E600009F0ADCF8091E2019091E3018D7F892B44
:101E700009F0A5CF8091E800877F8093E8008091EA
:101E8000E80082FF17C09091F3008091F200029762
:101E900031F48091F100813011F0863021F480918D
:101EA000F10080930F018091E8008B778093E80028
:101EB000B6DB85CF80914F028111E1CF80CF809139
:101EC000DE01813A09F07BCF8091E2019091E3013C
:101ED000892B09F074CF8091E800877F8093E80018
:101EE0008091E80080FFFCCF809110018093F10089
:101EF0008091E8008E77DACF8091DE01813209F09F
:101F00005ECF8091E800877F8093E80088DB809136
:101F1000E10180930E0153CF8091DE01813A09F0F7
:101F20004ECF8091E800877F8093E8008091E800A1
:101F300080FFFCCF80910E01D9CF803889F08238A4
:101F400041F58091E2018F70873018F58093E900A8
:101F50008091EB0085FB882780F91092E90006C08C
:101F600080912A02880F9091DB01892B9091E800E3
:101F7000977F9093E8008093F1001092F100809198
:101F8000E8008E7723C0811116C08091E001813076
:101F900009F18091E80083FF0AC08091E800877F03
:101FA0008093E8008091EB0080628093EB00AA961A
:101FB000E3E00C948833823061F78091E001811571
:101FC00081F01092E9008091E800877F8093E8001B
:101FD00026DBDFCF81E0933009F080E080932A0296
:101FE000F0CF8091E2018F702FEF280F263088F616
:101FF0008093E9002091EB0020FFE3CF933031F490
:102000008091EB0080628093EB00DBCF9091EB003E
:1020100090619093EB0021E030E0A90102C0440FF1
:10202000551F8A95E2F74093EA001092EA008091EA
:10203000EB008860E8CF8111ACCF1091E0011F77F1
:102040008091E3008078812B8093E3008091E80009
:10205000877F8093E800E3DA8091E80080FFFCCF7F
:102060008091E30080688093E30083E0111101C058
:1020700082E080934F028DCF8058823008F089CF64
:102080008091E0019091E1018C3D53E0950791F53D
:1020900083E08A838AE289834FB7F894DE0113963E
:1020A00020E03EE051E2E32FF0E0509357008491AE
:1020B00020FF03C082958F703F5F8F708A30C0F021
:1020C000895C90E08D939D932F5F243161F74FBF22
:1020D0008091E800877F8093E8006AE270E0CE019B
:1020E000019644DA8091E8008B778093E80051CF25
:1020F000805DE7CF292F33272330310509F44EC007
:1021000078F52130310509F488C08BE590E0EFE2E5
:10211000F2E02230310509F03CCF2091E800277F22
:102120002093E8002091E4013091E50182179307A4
:1021300008F49C0140E02115310509F073C04111FC
:1021400071C08091E80082FDCDCF80914F02811552
:1021500049F2853039F28091E80083FFF2CFC2CF97
:102160008091E2019091E3012132310509F446C0EA
:102170002232310509F00DCF8330910508F009CFE7
:10218000FC01EE0FFF1FEF5DFE4F0190F081E02D8F
:10219000825E9E4FDC018C9190E010C09C01332741
:1021A000823021F12330310568F4232BB9F4EAEDB4
:1021B000F2E0E4918E2F90E0EAEDF2E0009709F46E
:1021C000E8CEABCF2330310509F0E3CEECE9F2E005
:1021D000E4918E2F90E0ECE9F2E0F0CFEAECF2E04F
:1021E000E4918E2F90E0EAECF2E0E8CFEAEBF2E047
:1021F000E4918E2F90E0EAEBF2E0E0CF833091059E
:1022000008F0C7CEFC01EE0FFF1FE95DFE4F019005
:10221000F081E02D89E090E080CF82E190E0EAE873
:10222000F2E07BCF80914F02811509F45BCF8530BE
:1022300009F458CF8091E80083FD54CF8091E800E5
:1022400082FD7FCF8091E80080FF75CF9091F300F1
:102250008091F2002115310519F08830910550F078
:1022600041E0089709F040E08091E8008E77809384
:10227000E80061CF44914093F1003196215031093B
:102280000196E8CF803809F084CE8091E800877FFE
:102290008093E8008091DC018093F10070CE811181
:1022A00078CE1091E001123008F073CE8091E800F2
:1022B000877F8093E8001093DC01B1D91115D9F024
:1022C00084E080934F0242E061EC81E025DA42E253
:1022D00061EC84E021DA42E261EC82E01DDA42E264
:1022E00060EC83E019DA80914F02843051F482E08F
:1022F000809311014ECE8091E30087FDE1CF81E014
:10230000E0CF81E0F5CF80911301877F80931301A7
:1023100080911803811103C082E00E9479058091A9
:10232000130184FF06C08F7E8093130182E00E9418
:102330006B058091130185FF06C08F7D809313018B
:1023400080E20E946B0562CBCF92DF92FF920F93E7
:102350001F93CF93DF93EC018B01F42E8091130137
:1023600082FF61C0C0902704D0902804CC16DD06FF
:1023700019F0209709F057C0809113018B7F80934B
:102380001301C1E081FD10C08091250490912604C5
:102390009801281B390BC1E080910C0190910D012F
:1023A0002817390708F4C0E080911301C0FB81F9B8
:1023B000809313016C2FC6010E94700880913B042A
:1023C00081FF08C08091130180618093130182E036
:1023D0000E94710580913B0485FF08C08091130124
:1023E00080628093130180E20E9471056C2FC60108
:1023F000F3DBF11431F08091B20485FF02C086FF57
:1024000025C08091B5049091B6042FDA80912704FD
:10241000909128049C0130522115304308F49927EB
:102420000DDC71DF0FC0CE01905281159043B0F4E6
:10243000CE01992703DC8091270490912804C817C6
:10244000D90779F31093260400932504DF91CF91E7
:102450001F910F91FF90DF90CF900895CE01EACFAA
:10246000CF93DF93EC014A855B856E857F850E9463
:1024700004098B810E9479058C810E947105C6DA5E
:1024800086E0FE0111928A95E9F7DF91CF910895D8
:10249000CF93DF93EC018D8181FD13C082608D832A
:1024A00080913E049B81892B80933E048C810E9405
:1024B0006B05ACDA488559856E857F85CE010E9413
:1024C000040910922204109221048D8180FD02C023
:1024D000CE01C6DFDF91CF9108951F93CF93DF9395
:1024E000182FA0919703B0919803109709F449C051
:1024F00010929A031092990310921D0310921C03DC
:102500001696CD91DC911797CE019A9581159F4132
:1025100008F4D07ED1E0C11101C0D0E01996ED9150
:10252000FC911A97309731F01B966D917C9180E069
:102530000995D823D11539F08CEF8C0F813A28F505
:102540008C2F0E949C091115A9F0E0919703F0913E
:102550009803808584FD0EC080919603811551F00B
:10256000808191819C01215031092F333E4710F425
:102570000E94740A4BDA10929803109297031092FB
:102580009603DF91CF911F91089540DA8C2F32DBB3
:10259000DACF0F931F93CF93DF9307E914E0C9E5D8
:1025A000D2E0CE010E94CA33F80161918F01681711
:1025B00019F0CE010E94E6332196C138F2E0DF0720
:1025C00081F7DF91CF911F910F9108950F931F9382
:1025D000CF93DF9307E914E0C9E5D2E0CE010E9472
:1025E000CA33F80181938F012196C138F2E0DF07E9
:1025F000A9F7C0E0D4E0FE0185919591009711F014
:10260000FC0109952C96F4E0CC3CDF07A1F7DF91A3
:10261000CF911F910F910895E7E9F4E0128E138E88
:102620008FEA90E09183808385E0848F28E833E10E
:102630003383228322E330E0378B268B28EC30E093
:10264000318F208F158E35A324A3178E168E20E58B
:1026500030E031A320A382A317A216A29ADF24DBC5
:102660001092C0041092BF0480E084608093C00484
:1026700060E074E084E090E00E940034A7CF0F9304
:102680001F93CF93DF93843030F5653020F54E30C3
:1026900010F5C42FD0E0CC0FDD1F2CE1629FC00DE0
:1026A000D11D11243CE8839FC00DD11D1124CE0102
:1026B00089960E94CA33082F10E0102F0027CE0100
:1026C0008A960E94CA339801282BC901DF91CF91C5
:1026D0001F910F91089580E090E0F8CF462F672F6B
:1026E0002091520230915302232B81F4703F39F430
:1026F000403F61F4809150029091510208957530ED
:1027000028F44E3018F4843008F4B9CF80E090E01B
:102710000895A0E0B0E0EFE8F3E10C9468337C01A9
:1027200000913A0480913904082BC3E0D0E010E016
:10273000C8010C2E02C0959587950A94E2F780FD9A
:1027400009C02197A8F7D12C8D2DCDB7DEB7E7E0D2
:102750000C948433DC2EB7018C2FC0DF0E947F06DF
:10276000019779F3F1CFCF93DF93D82FC92FD1DF22
:102770006D2F7C2FB3DF0E947F06DF91CF910895EC
:10278000FC018481811561F087819085009721F09B
:102790000E947F060C940A0480819181E4DFFACFC5
:1027A00080E008951F93CF93DF93182FD92F6115E1
:1027B00089F0411579F0ADDFC82F682F812F9D2F4B
:1027C0000E944C04612F7D2F8C2F88DFDF91CF91E9
:1027D0001F9108950E948204C82FF4CFFC01462F58
:1027E00087819085009721F4658180819181DACF7E
:1027F0000895382F292FCB01A32FB22F8F3A91059F
:10280000A105B10520F48F5A9C4F0C94CA3380E087
:10281000089585E290E00E94CA33833089F486E20D
:1028200090E00E94CA33813459F487E290E00E941C
:10283000CA3391E0863909F090E0892F81700895BC
:1028400080E0FCCFAAE0B0E0E8E2F4E10C9462336F
:10285000C0904D02D0904E0281E090E090934E02E5
:1028600080934D02812C912C10E0540100E019C09E
:1028700021E030E0123020F4F701859195919C0120
:10288000472D602F812F9BD8739422E0E20EF11C1C
:102890003EE07312EDCF0F5F8EE0A80EB11C053045
:1028A00049F0C501880F991FFC01E252FD4F7F01DD
:1028B000712CDECF1F5FF6E48F0E911C1430A9F649
:1028C000ABDE1A8219821C821B821E821D82188630
:1028D0001F8288EC90E09A87898701E812E09E01C8
:1028E0002F5F3F4F79014AE050E0B801C7010E94D5
:1028F0000434065F1F4F013D32E01307A1F789E062
:10290000F70111928A95E9F78FEF9FEF9E838D83F0
:1029100087E08A874AE050E0B801C7010E9404348A
:10292000065F1F4F0132F3E01F07A1F786E0F701B2
:1029300011928A95E9F746E050E0B801C7010E947C
:1029400004340A5F1F4F0135F3E01F07A1F7D0924F
:102950004E02C0924D022A96EDE00C947E33AAE01E
:10296000B0E0E5EBF4E10C9465330EE113E081EDAA
:10297000E82E82E0F82E97E0B92E26E1C22E22E062
:10298000D22EAA24A3944AE050E0B701CE010196CA
:102990000E94BA33F8013896DF018B2D1D928A957B
:1029A000E9F789819A81D80111969C938E938F8142
:1029B00012968C9312978D8113968C93139788851A
:1029C00014968C931497898515968C9315978B8103
:1029D0009C8117969C938E9316978A8587FD04C0D9
:1029E0001E96DC92CE921D9780FF02C0F801A08651
:1029F00081FF07C0D80118969C911897926018968D
:102A00009C9382FF04C0F80190859460908783FFB7
:102A100007C0D80118969C911897986018969C93B7
:102A200084FF04C0F80190859061908785FF07C0FE
:102A3000D80118968C911897806218968C93BAE0FA
:102A4000EB0EF11C015F1F4FE1E2EE16E3E0FE0624
:102A500009F099CF2A96EAE00C948133A6E0B0E021
:102A6000E4E3F5E10C94683308EB12E081E2E82E30
:102A700083E0F82E98E0D92E46E050E0B701CE0171
:102A800001960E94BA33F8018D2D11928A95E9F7CB
:102A9000B8016C5F7F4F89819A810E94BB07F80162
:102AA00091838083B8016B5F7F4F8B819C810E94F3
:102AB000BB07F801938382838D8186838E81878310
:102AC000F6E0EF0EF11C085F1F4F81E5E81683E08A
:102AD000F80691F62696E7E00C948433282FCB0174
:102AE000283070F44AE0249F90011124B9016F57F7
:102AF0007D4F4AE050E00E94BA3380E090E00895B4
:102B00008FEF9FEF0895AAE0B0E0E9E8F5E10C94BB
:102B10006D339C0197558115914068F4BE016F5F3C
:102B20007F4F822FDBDF892B31F489859A852A96A6
:102B3000E2E00C9489338091AF049091B004F7CF18
:102B4000A0E0B0E0E6EAF5E10C946833162FD72F49
:102B5000C42FD22E8115A9F0409332040E94CB09D4
:102B60009093DA018093D901C77081E001C0880F8A
:102B7000CA95EAF70E945A0DCDB7DEB7E7E00C948C
:102B8000843390913204491336C0E090D901F0901B
:102B9000DA010E94CB099C012E193F097901812F8E
:102BA0009D2FB1DFE816F90630F5D0E2DD0DCD1529
:102BB000A1F0C77011E0812F01C0880FCA95EAF714
:102BC0000E94680DD83048F48D2D877001C0110F18
:102BD0008A95EAF7812F0E945A0D802F5AD8D83053
:102BE00058F62D2D277081E001C0880F2A95EAF74D
:102BF0000E94680DC1CFC77081E001C0880FCA95DF
:102C0000EAF7F6CF9C01CB01BA01F9013296E491C3
:102C10004E2F50E06E17710548F0F901349665911A
:102C200075910E94AA3380E090E008958FEF9FEFA6
:102C30000895A4E0B0E0EFE1F6E10C946A338B0173
:102C4000FC013396F49019821A821B821C82452B58
:102C500031F48FEF9FEF2496E5E00C94863344E047
:102C600050E0BE016F5F7F4FCDDF019691F381E0B1
:102C700090E00F2C02C0880F991F0A94E2F7092EEA
:102C8000000CAA0BBB0B49815A816B817C81842388
:102C90009523A623B72321E0892B8A2B8B2B09F4BC
:102CA00020E0F801208380E090E0D5CF9C01CA01AC
:102CB000F9013296E4914E2F50E08E17910550F0B5
:102CC000F9013496859195910E94AA3362DC80E0E7
:102CD00090E008958FEF9FEF0895A4E0B0E0E3E760
:102CE000F6E10C9466337C016B01CA01F70133965F
:102CF000B49019821A821B821C82892B31F48FEFC7
:102D00009FEF2496E9E00C94823344E050E0BE014A
:102D10006F5F7F4FC70176DF019689F381E090E016
:102D20000B2C02C0880F991F0A94E2F780959095AA
:102D3000092E000CAA0BBB0B49815A816B817C8147
:102D400084239523A623B723F6012081022F017047
:102D500010E00B2C02C0000F111F0A94E2F7012EA5
:102D6000000C220B330B802B912BA22BB32B8983CE
:102D70009A83AB83BC8344E050E0BE016F5F7F4F1A
:102D8000C70194DFBECFAAE0B0E0E9ECF6E10C9415
:102D90006133FE0131968AE0DF011D928A95E9F7E1
:102DA0009DE2A92E91E0B92E8F013F01EE24E3941C
:102DB000F12C30E4C32E31E0D32EF50181915F0177
:102DC0008F3F09F444C0F894E82FE295EF70F0E0EB
:102DD00021A18F70A70102C0440F551F8A95E2F709
:102DE000CA01922F982B91A392A18095892382A347
:102DF000789400C0E2E3F1E021E030E0812C912CF6
:102E000041914F3F79F0A42FA295AF70A05EB0E042
:102E10008C9190E04F7002C0959587954A95E2F7A6
:102E200080FF3BC080E090E0882A992A220F331F60
:102E3000CE16DF0629F7F50182918F3F11F00E942F
:102E40007D0750EA5A95F1F7D8018D929C920E5F5A
:102E50001F4FB2E3AB16B1E0BB0609F0AECF4AE0BC
:102E600050E0B3018FE192E00E949D33892BB9F0CD
:102E70008AE0F301AFE1B2E001900D928A95E1F7AB
:102E800081E08093D8010E94CB099093D701809371
:102E9000D6012A96EEE00C947D33C901C5CF80910E
:102EA000D8018115B1F30091D6011091D7010E948C
:102EB000CB09801B910B059760F34AE050E06FE16E
:102EC00072E083E492E00E949D33892B49F08AE00E
:102ED000EFE1F2E0A3E4B2E001900D928A95E1F710
:102EE0001092D801D6CFA0E1B0E0E9E7F7E10C9469
:102EF0005F33FE01319680E1DF011D928A95E9F78B
:102F00000BE010E091E5A92E93E0B92E2FEA422EB6
:102F1000512C612C712C4F0173016201B1E14B16F0
:102F20005104610471041CF080E1C82ED12CA6016B
:102F3000B501C4010E94D733AC0CBD1C0D2C000C94
:102F4000EE08FF084C185D086E087F08015010401D
:102F500019F76096E0E10C947B336FEF85E290E027
:102F60000E94E6336FEF86E290E00E94E6336FEF57
:102F700087E290E00E94E63360E088E290E00E9401
:102F8000E63360DCB0DF63E085E290E00E94E63388
:102F900061E486E290E00E94E63366E987E290E031
:102FA0000C94E633A0E0B0E0E8EDF7E10C94663372
:102FB000EC0188818115F1F0813009F042C08981EE
:102FC000813029F48A8123960E94490EF2CF823003
:102FD00029F48A8123960E947B0DEBCF833029F45C
:102FE0008A8123960E94FA0DE4CF843041F0229624
:102FF0008111DFCFCDB7DEB7E9E00C9482338A814F
:10300000239620E030E09AE0682F6053770BAB0105
:103010006A30710560F02115310551F3EFE9FFE0E9
:103020003197F1F700C0000021503109F4CF929F91
:10303000B001939F700D11249A01260F371F8991BB
:10304000E3CFE82FF0E0E155FE4FB490282F26950E
:103050002695269530E0F901E156FE4FE490877001
:10306000F12C082E02C0F594E7940A94E2F7E0FAF6
:10307000EE24FF24E0F8F901E157FE4FC490D12C73
:10308000082E02C0D594C7940A94E2F7C0FACC2463
:10309000DD24C0F8F901E158FE4F049110E002C0B0
:1030A000159507958A95E2F701701127E114F1044F
:1030B00019F081EE0E947B0DC114D10419F086EE47
:1030C0000E947B0D60E070E08B2D0E94330EC114D6
:1030D000D10419F086EE0E94FA0DE114F10419F002
:1030E00081EE0E94FA0D0115110519F08CE20E9483
:1030F000490E21965ECFAEE0B0E0E1E8F8E10C9435
:103100005D337C01DC0114968C91811509F4BCC1FE
:1031100060E0C70163DB9C01F7018681803170F4B8
:103120004091450490914404491333C09091930415
:10313000911521F090919404903158F1D701159692
:103140009C91911110C02115B0E53B0708F084C097
:103150002115E0E23E0708F094C0283E310590F4C6
:10316000203E3105B0F43093AD022093AC02D7017C
:1031700012968D919C9190934304809342041092F7
:10318000140107C0C9019A9581159F4160F721116B
:10319000EACF61E0C70122DB8C01F701858181154F
:1031A00021F180912104909122040097F1F00817F9
:1031B0001907D9F0FC01FF27887F9927892B09F08F
:1031C00062C084E0EE0FFF1F8A95E1F7EF55FC4FD8
:1031D00085818460858311830083CF0159D9109242
:1031E0003E0461E0C701FADA8C0180910D03811180
:1031F00051C0D70115968C91811509F4FBC00115BA
:10320000B0E51B0708F0E1C00115E0E21E0708F079
:103210003FC10115F7E01F07E9F1C0F5C801805E65
:1032200091090897B8F130913B0480913E042091B8
:10323000370499E0F701A9EFB2E001900D929A9559
:10324000E1F7109301030093000310920303832B13
:10325000822B8093F8021EC0203E42E5340760F4C2
:10326000203852E5350708F094CFC90180529245C5
:10327000809708F078CF8DCFC90187579C47029778
:10328000F8CF8031F6CFE0E0F0E0A2CF01153FE0CB
:10329000130749F6F70185818111F7C1011527E56B
:1032A000120708F401C3011538E5130710F00C9458
:1032B0009724680147E5D41A6EE073E08C2D0EDC8C
:1032C000892B31F5C601F4E0880F991FFA95E1F7D3
:1032D000FC01EF55FC4F2281213009F0B5C220914D
:1032E0000E0330910F03232B99F02091100330919E
:1032F0001103232B69F020911203309113034091A5
:10330000140350911503242B352B232B09F4A6C24B
:1033100080911803811509F441C3C0903B04D090FB
:1033200037040E94CB0988579C4E90931A038093D0
:103330001903D70115968C91811509F42FC38D2D92
:103340008C298D79811153C30115B0E51B0708F055
:1033500001C30115E0E41E0708F050C3063E110545
:1033600009F41CC3C80190528115904208F007C3AC
:10337000D70116968C91803108F433C36801DD249F
:103380008091130180FF46C38DEF0E947905BDE255
:10339000CB16D104A1F008F050C3F8E2CF16D10447
:1033A00008F03AC32EE1C216D10408F039C334E064
:1033B000C31AD1084AE1C416D10408F018C3809199
:1033C0003E04826080933E042BC3003E42E5140716
:1033D00050F4003652E5150708F05CCFC80192554D
:1033E000803491051FCF980127573C472530310580
:1033F00008F019CF0937BCE71B0709F04EC0209130
:10340000000330910103232B79F18115A1F081E0B4
:103410000E94DE088091F8020E945F0D89E0E9EFCA
:10342000F2E0AFEAB2E001900D928A95E1F7809167
:1034300003038093AE0286E0F701AFEAB2E00190A9
:103440000D928A95E1F78091AE0280930D038FEA89
:1034500092E051DE10920D03F7018581811104C0C5
:103460008091F8020E946D0D80913F048770811554
:1034700059F0F7018581811539F08091C00482FFF0
:1034800003C082E00E9450052E96E2E10C9479334D
:10349000D70116968C918031C5CE0A37FCE71F07FD
:1034A00009F0F8CE811509F4C5C0A0900003B090D2
:1034B00001032091F8022F832983BE016F5F7F4FA4
:1034C000C5010E94BB072C0139813D87B8EBCB2E8B
:1034D000B2E0DB2E01E010E022242A94D6011796F8
:1034E0003C90179733FE53C06D907C9011971296C5
:1034F0008D909C90139746145704B9F41496BC9180
:10350000BB87232DF60146816B2F8D850E94D50741
:10351000811559F08B850E94F403281634F4D601E6
:1035200015969C918401192B282E48145904C9F42E
:1035300031FE17C0F601F581FB87232DD6011696C3
:103540004C916F2F8D850E94D507811551F08B8589
:103550000E94F40328162CF4F60194818301192BA0
:10356000282E30FE14C0FFEF2F1211C001301105BC
:1035700071F4232DD60116964C9160E08D850E9442
:10358000D507811521F0F60185818401182BF8E01B
:10359000CF0ED11C28EF32E02C153D0509F09ECF4F
:1035A00001301105E1F58F8182958F703F81832B6A
:1035B0008F7011E0303108F410E01295107F182B55
:1035C000A11440E2B40620F5A11451E0B50608F0BC
:1035D00055C00A2D812F8D704A2D811509F451C0D7
:1035E0006AE086E097E00E94EF08282F30E021157E
:1035F000310551F4402F66E188EE96E00E94EF0815
:10360000282F30E0811549F0F901F12B8F0107C017
:10361000C50190528115904390F100E010E087E0E1
:10362000E4E0F3E0DF011D928A95E9F710930C03C3
:1036300000930B0380910B0390910C03892B09F4E9
:1036400013CFF7018581811539F08FEF0E94DE08D5
:10365000809103038093020386E0F701A4E0B3E0C6
:1036600001900D928A95E1F78091020380930D03FA
:1036700084E093E040DD10920D03F6CE1B29BB24BD
:10368000A8CF68E08EEF96E0AECFC801975780389C
:10369000910508F0EEC0003108F0E6CE6EEA70E069
:1036A00080E090E0A6D88111DFCE812C912C5401CE
:1036B000011143C004E0AE014F5F5F4F6A01D601C4
:1036C000E02F1D92EA95E9F724013501FFEF4F1A2B
:1036D0005F0A6F0A7F0AC501B4018BD889838115FF
:1036E00009F4C2CE813009F0ACC0A50194012E5F6F
:1036F0003F4F4F4F5F4F2F83388749875A87C3010A
:10370000B20177D8182F8A83811509F4ADCE8FEFD7
:10371000810F833050F56F81788589859A8569D8C6
:103720008B83811511F0C6013DDC2401350133E0A6
:10373000430E511C611C711C46C0FFEA8F16910498
:10374000A104B10409F490CEC501B40152D82FEF01
:10375000821A920AA20AB20A8111EFCF0150A8CFB1
:103760004F80588469847A842EC08BEF810F833018
:1037700098F52401350143E0440E511C611C711C75
:103780006F81788589859A8534D88B838115D9F0A6
:10379000C301B2012ED88C83811571F08B819C817D
:1037A00081305FEF950710F0982F8827163071F061
:1037B000173079F00E94392A2401350154E0450E72
:1037C000511C611C711C5301420179CF0E94F729E1
:1037D000F3CF0E94182AF0CF143009F0C1CF6F81C7
:1037E000788589859A8505D8182F2401350184E0CC
:1037F000480E511C611C711CC501B4016D5F7F4FE7
:103800008F4F9F4F0E94F913111509F42DCE81158A
:1038100009F42ACE8150990B4FEF489F9001499FA0
:10382000300D1124A12FA150BB0B2A0F3B1F21509B
:10383000310948F2EFE9FFE03197F1F700C00000ED
:10384000F6CFC601AFDBBFCF223009F061CD2091AA
:10385000120330911303232B09F45ACDFC01EA55CE
:10386000FC4F20812E7F20838F559C4F0E94481251
:103870004FCD03375CE71507B9F480911803811524
:1038800019F00E94720DF0CD10923B040E94810548
:103890000E94CB0988579C4E90931A03809319037A
:1038A00081E080931803E0CD023A82E51807C1F168
:1038B00058F4C80190528115904220F1013E110543
:1038C00079F1053E110503C0023BB2E51B0709F083
:1038D0001FCD25EE30E02770332781E090E001C056
:1038E000880F2A95EAF720911B03309118033115B0
:1038F000F9F0D70115963C913115A9F0282B2093AA
:103900001B03B2CDF7018681803108F001CD812FF4
:1039100099278F7199278230910511F04297D7CF5F
:1039200021EE30E0D8CF8095822380931B039CCD7D
:10393000322F3823311509F4EBCC982F9095922330
:1039400090931B030E947105F7018581811509F48D
:103950008BCDDECC003EB2E51B07C0F4003CE2E5B7
:103960001E07E0F4003AF2E51F0758F4003622E59E
:103970001207A0F4C80192558034910578F06801CF
:10398000FFCC043B32E5130749F0F9CF09374CE788
:10399000140718F507375CE7150788F3D701159664
:1039A0003C90311409F456C00E35BCE71B0709F4EE
:1039B0004DC00F35ECE71E0751F00D35FCE71F0732
:1039C00009F048C080911201811509F43FC010929E
:1039D000120180E00E946D1247CD0B378CE718076B
:1039E000D3CF812F8F718431C9F2863171F00E945B
:1039F000720D80911B030E946B05D0CFD7011696E4
:103A00008C91803108F0BACCC9CF76EEC72E72E126
:103A1000D72EB6CC8FEFB9CC5AE2C516D10439F700
:103A200080911B03811531F080913E0492E089273B
:103A300080933E040E94060DB1CF8CE4C816D104D9
:103A400079F39DE2C91692E0D906E9CF81E080932F
:103A500012010ACD80911201811149C0C801975508
:103A60008115914008F0DFC05801F8EFAF22BB2468
:103A7000A114B10409F0F8CCF801FF2754E0EE0FCF
:103A8000FF1F5A95E1F79F012F553C4F6901D70160
:103A900015968C91EA55FC4F908180FB90F99083AC
:103AA000811509F412C20E94CB09909324048093DB
:103AB0002304F60182818F5F828380913E0490917E
:103AC0003B04892B8383809137048483468157810B
:103AD00066857785C6010E940409D60115968C91EA
:103AE00081FF5801B0922204A09221049CC03801A9
:103AF00030EE631A71085090380480913B04582AC4
:103B000080913704582A48E06416710408F05EC0BA
:103B100098012770332781E090E001C0880F2A9533
:103B2000EAF7311409F44FC0582AD7018D919C91BE
:103B30000E94820421E030E0F90102C0EE0FFF1F75
:103B40008A95E2F7FC87EB872091970330919803E1
:103B500038872F8340919F035091A0035E874D8744
:103B60006EE1C62E63E0D62EA12CB12C511005C0FB
:103B7000D60112968C9181111BC0F601838190E0D1
:103B80002B853C8582239323892B91F08085982F68
:103B90009770911101C087E038E06316710408F056
:103BA000BFC0311409F4B8C0869581708111BDC0C1
:103BB0009FEFA91AB90AAFE0CA0ED11CB8E0AB1644
:103BC000B104A1F61CC080955822AFCF311091C02E
:103BD00080919F039091A0030817190781F4109218
:103BE000A00310929F0310929B0310929C031092CB
:103BF0009D0310929E0310929A0310929903809154
:103C0000970390919803009709F428CFE8E06E1687
:103C1000710408F044C1652D0E949608811103C00B
:103C200081E00E946D128091B20480FFBEC10E94AB
:103C3000CB095C01F7018581811509F4C8C1809128
:103C4000130182FF06C040E0B50180E090E00E94D1
:103C5000A4110431FCE71F0709F4B5C105312CE7B5
:103C6000120709F44FC103313CE7130709F490C16F
:103C7000C80190528115904308F04EC1109228045B
:103C800010922704F70195819111109232040631A8
:103C9000FCE71F0709F06EC280913B043091B1042C
:103CA00030FF04C0282F2474211158C2282F2A7AEB
:103CB00031FF04C0482F4171411120E032FF04C0A0
:103CC000482F4878411120E033FF03C082728111F0
:103CD00020E0911509F444C281E0211101C080E087
:103CE0008093330485E3211101C089E20E946809B1
:103CF000C7C01093A00300939F030E94680A6093BB
:103D00009B0370939C0380939D0390939E0310925A
:103D10009A031092990309CF82FB882780F946CF36
:103D2000311409F445CF80FF43CFD6018D909C908C
:103D30000815190519F4311409F43ACFEF81F88503
:103D4000EC15FD0509F434CFD6011D96ED91FC91DB
:103D5000309721F08081811509F42ACF652DC601A5
:103D60000E949608811509F423CF81E008151905F2
:103D700009F080E0482E43208114910441F0411065
:103D800006C0ED85FE858E169F0609F011CF80E0F6
:103D90000E946D12D0929803C092970381E08093A5
:103DA00096038FE08A9DF0018B9DF00D1124E25E59
:103DB000FC4F858180931D0341100EC08114910436
:103DC00059F0808191819C0124503109213A3105BB
:103DD00008F049C00E949C098FE08A9DF0018B9DEC
:103DE000F00D1124E25EFC4FC680D780C6019A9583
:103DF00081159F4110F420EED22299249394C6019C
:103E000001978F339E4708F0912C8FE08A9DD00157
:103E10008B9DB00D1124A25EBC4F1996ED91FC91C3
:103E20001A97309731F01B966D917C9181E009953E
:103E300098229114A9F08FE08A9DF0018B9DF00DDE
:103E40001124E25EFC4F868197810E94C10380931A
:103E50001C03C60148E06416710440F40E94740A11
:103E60000E94060D0AC00E94FA0DB6CF0497813A4F
:103E7000910548F48C2D0E946809411409F4EECD97
:103E80000E94060DF1CA0E94060D8FE39CE901977E
:103E9000F1F700C000008C2D0E947B0DEECFDC01FD
:103EA0002D913C910217130741F4311009C0109273
:103EB000960380E00E946D12D1CD311409F4CECD6D
:103EC000FC01808585FDCACDF4CFF9014485558577
:103ED00066857785C9010E940409D60115968C91E3
:103EE00081FFA1CEC6010E943012809121049091E1
:103EF00022040817190709F096CE10922204109296
:103F0000210491CE90911301892F8E7F90FF8160C3
:103F1000809313010E9483118091130180FF45C09B
:103F20000832110508F069C00E31110508F076C09D
:103F3000C80104974A9788F58091B20484FD2DC08A
:103F4000D70115968C91811509F4D6C0809137045C
:103F500090913B04892B8D7F811509F464C01092E8
:103F60002804109227048091B20481FD5CC060E0B7
:103F7000C8010E94700860E0C8010E94EC0D8091A9
:103F800037048D7F0E94550A82E00E9450056CCA5A
:103F900080911301816080931301F7018581811560
:103FA00021F01092280410922704D70115968C91C5
:103FB000F801E851FC47E730F10508F063CEE95D10
:103FC000FB4C0C944033809113018E7FA1CF8091E4
:103FD00013018F7E013E110531F0053E110531F4CC
:103FE000809113018F7D8093130196CFC801905269
:103FF0008115904308F090CF45CE0933110558F450
:104000000D32110518F40B32110539F68091B20406
:1040100082FDC3CF95CF04361105F7CF8091B2044E
:1040200083FDBBCF8DCF89E0F701A9E2B4E0019019
:104030000D928A95E1F710922C0410922B04809136
:1040400027049091280408171907C9F52091B20494
:1040500025FF35C03091130131FF02C026FF2FC06C
:1040600020912504309126046501C21AD30A0E94CA
:104070008315C816D90618F580913B0481FF08C046
:104080008091130180618093130182E00E94710589
:1040900080913B0485FF08C080911301806280936A
:1040A000130180E20E9471056091130166956170B1
:1040B00080912704909128040E94EC0DD5C980912D
:1040C0003704D0903B04D82AD1FADD24D0F88D7F74
:1040D0000E94550A1093280400932704B0922604E6
:1040E000A0922504DD0C6894D2F890911301997F79
:1040F000D92AD092130148CF40E0B501C8010E94EF
:10410000A411B2C906E221EE41EE6AE17CE70E9409
:10411000A015AAC907E225EE45EE6BE17CE7F7CFD3
:1041200006E221EE40EE68E17CE7F1CF07E225EE02
:1041300044EE69E17CE7EBCF06E221EE42EE6CE172
:104140007CE7E5CF07E225EE46EE6DE17CE7DFCFC9
:1041500008E221E045EE6EE17CE7D9CF20E0A8CD72
:1041600080913304811521F085E30E949C0988CE5B
:1041700089E2FBCF07372CE71207F9F008373CE755
:10418000130731F19801205E32452032310528F5C0
:10419000911123C00F7181E090E0AC0102C0440F87
:1041A000551F0A95E2F78A01642F83E090E00E9490
:1041B000E633802F0E942E0457C981E0911551F0FB
:1041C0000E94340443E062E081E00E94B6044CC9DE
:1041D00082E0F4CF0E943E04F5CF409134048091F8
:1041E0003A04282F30E02095309570E024233723BF
:1041F000232B19F04823409334040B375CE7150751
:1042000041F4911509F430C90E94F7030E94B708E0
:104210002BC9003482E5180708F056C00032A2E529
:104220001A0708F058C00115B0E51B0758F501152D
:10423000E0E41E0708F065C0911509F47BC00A355B
:10424000BCE71B0709F4FBC008F0DFC00130FCE746
:104250001F0709F4F2C003302CE7120709F4E7C086
:1042600001153CE7130709F065C00E94540E8FEF5B
:1042700094E3ACE081509040A040E1F700C0000022
:104280000E94430C9801305521153240A8F6980140
:1042900045E0369527954A95E1F7822F8F7020915A
:1042A000340430E041E050E0082E02C0440F551FB6
:1042B0000A94E2F724233523232B09F4BDCF91116F
:1042C000A5CF10923B04DCCD9801205C3245203212
:1042D000310508F0B1CF802F8F712091340430E088
:1042E00041E050E0082E02C0440F551F0A94E2F747
:1042F00024233523232B09F49FCF911509F4B4C847
:1043000085CFD70116968C91803108F095CF911109
:1043100011C0212F2F7081E090E002C0880F991FFB
:104320002A95E2F72091340430E082239323892BED
:1043300009F09AC8D70117968D919C91009709F4BE
:1043400082C00E947F06082FD92E86E0F701DE0189
:10435000119601900D928A95E1F7D7011596BC90C0
:1043600015971696CC90C2949FE0C92280913F0485
:104370008770811501F19B2CB114F1F08D2D807F98
:10438000803461F080E2800F8830A8F08D2D807E2F
:10439000803221F4023078F0C11469F08091C004B9
:1043A00082FF09C082E00E94500580913F0487701F
:1043B000992493948111912CAD2CA2948FE0A82282
:1043C000B8E0AB1609F481C1E9E0AE1608F08BC085
:1043D000F4E0AF1608F04FC01D2D1F7022E0A216AA
:1043E00008F494C08D2D807F803211F01295107FDB
:1043F000011509F4BFC0013009F429C1B11409F451
:1044000035C1C11409F4D0C095C00B354CE7140771
:10441000C1F08091C004002482FF0394802D0C35EC
:104420005CE7150709F086CF0E94C90C83CF6FEFB8
:104430007FEF80E090E00E9400340E94720E81E0E5
:10444000F3CF80E0F1CFF7018581C080D180811565
:1044500069F0C6010E948913182F682FC6010E94B7
:104460004C04B601812F0E946E136BCFC6010E94CF
:104470008204182FF6CF34E0A31609F409C1AA2D3F
:10448000A850BB0B149718F40E940909912C802F97
:104490009D2D0E940A04811541F0B11409F41CC23B
:1044A000C11409F410C21092C3049114B1F08091A8
:1044B0003F0480FD12C0D70115961C928695869503
:1044C00086950E943404C7010E947B1880913F04A6
:1044D0008695869586950E943E0460E0C7010E94FD
:1044E000EE130C94441A49E0A41609F45DC186E069
:1044F0008A0D8F70823018F6023F09F065C18D2D4C
:104500008F71B1105EC10E943404B9CF50E1D5164D
:1045100010F01295107FB114B9F0111559F080E226
:10452000800F883010F0011109C0812F0E946B05A7
:104530000E94060D802F0E947B0DA1CF80913E042A
:10454000812B80933E04F4CF802F0E94FA0D111529
:1045500009F495CF80E2800F883010F0011104C07B
:10456000812F0E94710503C0812F0E9479050E944E
:10457000060D85CF8091C00482FD12C0B11449F0B0
:10458000111529F0812F0E946B050E94060D80E015
:10459000D2CF80E00E94FA0D111509F470CFE0CF60
:1045A000B11491F1C11004C0812F0E945A0D67CF40
:1045B000B1E0CB1211C080903704812F88211817E9
:1045C00009F45DCF0E94CB099093360480933504A3
:1045D000812A8092370453CF8091B304823008F44B
:1045E0004ECFC8124CCF812F0E945A0D812F0E94AE
:1045F000400A80913804912F9823191709F43FCF6E
:10460000812B809338043BCFC11012C0812F0E94B0
:10461000680D812F0E94400A80913804912F9823C1
:10462000911509F42CCF109518231093380427CF37
:104630008091B304823008F422CFE1E0CE121FCF84
:1046400080913B048123811509F419CFDFCF80913C
:10465000B904B11421F08C1508F411CFA5CFC816F8
:1046600008F00DCF812F0E94680D09CFC114D1F33E
:104670008091B7049091B804093321F08091B5047A
:104680009091B6040E94350C802F0E94FA0DF7CE4F
:104690008D2D869586958370811569F0813009F09E
:1046A000EECE802F9D2D9370B11002C080E090E07F
:1046B0000E944009E4CE802F9D2D9370B11002C05E
:1046C00080E090E00E941809DACE8D2D8370811170
:1046D00033C0B110D4CE402F429546954770440F59
:1046E000440F802F8F70042E01C0880F0A94EAF7C0
:1046F000202F207104FF07C02FE030E001C0220FFF
:104700004A95EAF720953D2D36953695337032302F
:1047100071F0333051F040913904313029F0822B5F
:1047200084230E942E04ABCE842B822BFACF822BC3
:10473000909139048927F5CFB11459F1D0FE9FCE5D
:10474000402F429546954770440F440F802F8F703D
:10475000042E01C0880F0A94EAF7202F207104FF6D
:1047600007C02FE030E001C0220F4A95EAF72095FC
:104770003D2D369536953370323089F0333069F0FF
:1047800040913A04313041F0822B84230E9431045D
:1047900076CE8230A8F673CE842B822BF7CF822B75
:1047A00090913A048927F2CF1D2D1F70B11429F082
:1047B000812F0E943404802FF8CE802F0E94680D34
:1047C000812F0E943E045BCE60F4003FB9F0013FB0
:1047D00081F0B11409F472C0C110ACCE8D2D8F716F
:1047E00092CE033FF9F0043FA1F78091C00482FD0F
:1047F00025C08D2D8F71B11421F385CE8091B90420
:10480000B11461F0C81608F03ACE2D2D2F7181E059
:1048100090E001C0880F2A95EAF7C2CF8C1508F402
:104820002ECEF3CF80E0B11409F4B0CF81E09D2DFE
:104830009F7101C0880F9A95EAF7A8CF8091B304C1
:10484000823048F1B114C9F090913F0497709430D0
:1048500059F410923F0410924104109240048D2D9F
:104860008F710E943E0410CE63E0C81608F00CCE93
:104870008D2D8F710E942C0A07CEC81640F0109221
:104880003F04109241041092400464E0F1CF81E0B3
:104890000E945005F9CDB11431F063E08D2D8F7178
:1048A0000E942C0AECCD81E00E945005F2E0CF1668
:1048B00008F4E5CD82E00E945005E1CDC110D8CECC
:1048C0008D2D8F717ECF80913D0480933C0480912B
:1048D0003B0480933D04E9CD40E060E089819A810A
:1048E0000E94D2139C0110913B04C11429F0109234
:1048F000C30410933D04D9CD8091C1049091C204AA
:1049000028173907B1F78091B40482FFF0CF809166
:10491000C304811561F380913C040E945A0D802FDD
:104920000E94490E80913C040E94680DE0CF03373D
:10493000BCE71B070CC8A0E0B0E0E1EAF4E20C948D
:10494000683380919404803108F049C080919304C9
:10495000811509F444C0C091450489E0D82E8091A6
:1049600044048C17E1F1EC2EF12CDC9EE0011124C3
:10497000FE01EA5BFB4F84818115B1F19181809149
:104980008F04981331C0908180918E0498132CC0AD
:104990008581811129C002811381809190049091B9
:1049A0009104081B190B60E08EE894E00E94EE135E
:1049B0000E94831508171907B8F4809194048F702A
:1049C000806180939404C45BDB4F88818F70806129
:1049D00088838EE894E00E947B180E944605CDB73C
:1049E000DEB7E7E00C948433E7012196C770B7CFB8
:1049F000CF92DF92FF920F931F93CF93DF93182FE5
:104A0000092F89E0F82EC091450480914404C8170D
:104A100099F1FC9EE0011124CE018A5B9B4F6C0151
:104A2000FC018581811589F0C6010E94C0138115A2
:104A300061F0FE01E45BFB4F20812F702061208339
:104A4000F601808191810E94870EC6010E947B1829
:104A50002091450430E02F5F3F4F2770332720938C
:104A60004504CA5BDB4F89818013CDCF88818113D8
:104A7000CACF8D81811539F2DF91CF911F910F91AE
:104A8000FF90DF90CF900895EF92FF921F93CF9306
:104A9000DF93EC0120911401211541F010E0812FEA
:104AA000DF91CF911F91FF90EF900895EA80FB80F6
:104AB000E61AF70A24EFE21621E0F20678F760E042
:104AC000CE010E94EE139C0130522115304330F785
:104AD0000E941105811511F38091AC029091AD02F5
:104AE0000E941105182F8115C9F28091BD04909183
:104AF000BE04853F21E0920710F084EF91E0E816B4
:104B0000F90660F68E818F7080618E83888199812D
:104B10000E94870E0E94D504CE010E947B18BFCF51
:104B2000AFE0B0E0E6E9F5E20C945E338C0186E09C
:104B3000F801DE011A9601900D928A95E1F7D801ED
:104B40004C9011963C9011971296ED90FC90139713
:104B500014965C90149715966C9061100CC050914F
:104B60009002252F30E0E0E08E2F0E2E000C990BE6
:104B7000821793073CF15EE8A52E54E0B52E809194
:104B80009204811151C05114D1F0611409F419C378
:104B9000C8010E94C013811509F413C36091420437
:104BA00070914304C80170DF811109C089E0F801E8
:104BB000AEE8B4E001900D928A95E1F7BCDEFF24E7
:104BC000F3948CC0880F991F80589D4FDC0111967B
:104BD0004C911197431103C08C91481611F0EF5F6F
:104BE000C3CFEF3F41F2D80116968C9116978F7084
:104BF000806116968C93E517A0F4AFEFA50FA093F4
:104C00009002EA1770F4F0E0EE0FFF1FE058FD4F3E
:104C1000B0E0AA0FBB1FA058BD4F8D919C9191830E
:104C200080830E94D504A7CF60E08EE894E00E94C4
:104C3000EE136C0170909304809190049091910414
:104C40004701881A990A60E08EE894E0711409F42B
:104C50005CC20E94EE130E9483158816990608F024
:104C60000FC2511409F4ABCF80918F04F8019181E8
:104C7000B0909404F0E1BF1608F0C8C1981350C07A
:104C800090918E04D8018C9198134AC0611048C04D
:104C90008B2D8F708061809394048EE894E00E9445
:104CA0007B1880919404F8018683F0909004E09042
:104CB000910449E0D42E00914504809144040817E2
:104CC00051F0D09E800111240A5B1B4FD80115962C
:104CD0008C91811108C00E944605F12C8F2D2F96D2
:104CE000E1E10C947A33F801B280C380C8010E94DC
:104CF000C01381110EC0C8010E947B188091450429
:104D000090E001968770992780934504FB2CEC2C4A
:104D1000D2CF6F2D7E2DC801B7DE8111EFCFDBCF53
:104D2000F0E2DF1AC11420E3D20608F084C061105B
:104D300005C140E0632D842D0E94160C81114FC0E7
:104D400040E0632D842D0E94160CF82E811509F485
:104D500029C18091B40480FFC0CF8EE894E00E9406
:104D60007B1860E08EE894E00E94EE138C01F090D6
:104D700045047F2C98E0E92E2EE8822E24E0922E26
:104D800039E0432E809144047816A1F0A72CB12C71
:104D9000479CC0011124FC01EA5BFB4F6F0160E0FE
:104DA000CF010E94EE13582E692ED60115968C91D4
:104DB000811197C0B8E0EB1618F419E0EF10ACC001
:104DC0008A859B8515DE0E94D5040E94460589E0F0
:104DD000EEE8F4E0DF011D928A95E9F77ECF60E00E
:104DE000C8010E94EE138091B40483FFA9CFB801DB
:104DF0008EE894E00E94E2048111A2CF8091940495
:104E00008F7080618093940480918E0490918F04C0
:104E10000E94870E8EE894E00E947B18EEE8F4E092
:104E200089E0DF011D928A95E9F78A859B85E0DD9F
:104E30000E94D50450CF611409F482CF809194046C
:104E40008160809394048091B40481FF46CF8EE802
:104E500094E00E947B180091450480914404081757
:104E600009F4CCC0E02EF12CB9E00B9FC001112455
:104E7000FC01EA5BFB4F6F01CF010E94C01381155B
:104E800009F4BCC089E0F601AEE8B4E001900D92EF
:104E90008A95E1F7C701019687709927082F8093BB
:104EA00045040E94460589E0F82E8091440480174D
:104EB00009F411CFF09E800111240A5B1B4FC80139
:104EC0000E94C013811107CFC8010E947B188091F6
:104ED000450490E0019687709927082F8093450438
:104EE000E4CF10520115E0E31E0708F063CF809174
:104EF000B40483FD0AC0E72CC5010196F82FF770B2
:104F00007F2E052D162D46013DCFB601C4010E940E
:104F1000E204811589F3EFCF1F9DC00111248A5B44
:104F20009B4F0E947B182091450430E02F5F3F4F3C
:104F300027703327F22E2093450440CF80919404AC
:104F400081608093940460E0C8010E94EE13809118
:104F5000B40483FF78CFB8018EE894E00E94E204A5
:104F6000811171CFF0909404E894F0F8F0929404D9
:104F7000C8010E94C0138111B0CE8F2D8F70806147
:104F80008093940480918E0490918F040E94870EE8
:104F90000E94D5048EE894E00E947B18EEE8F4E0CD
:104FA00089E018CF8A859B850E94B313292F22950B
:104FB0002F70903450F49F70223080F0911599F04A
:104FC000F8019681903178F489CE2A5F2F702230D3
:104FD00078F0C8010E947B18F72C80CE911519F04B
:104FE000811509F47BCE805E883008F477CEF1CF4E
:104FF000803F08F473CE815F8330F7CF89E0EEE81D
:10500000F4E0DF011D928A95E9F74DCF981315C0A2
:1050100090918E04F801808198130FC061100DC02B
:10502000B682C8010E947B1889E0F801AEE8B4E0BE
:1050300001900D928A95E1F7C2CDC8010E94C0137C
:10504000811509F4BEC0611409F4BBC080919404B9
:10505000803208F4ABCD1E821F821886198680919B
:105060008E0490918F049A838983FC82EB828091D5
:1050700092048D83BF82CE0101960E947B1896CD4B
:10508000D0909404F0E1DF1638F48EE894E00E94AA
:105090007B1889E0D5019FCE511409F490CD9091F1
:1050A0008F04F8018181981311C090918E04808142
:1050B00098130CC061100AC0D682C8010E947B18E8
:1050C00089E0D5011D928A95E9F779CDC8010E9442
:1050D000C013811509F475C0611409F472C0809180
:1050E0009404803208F462CD1E821F8218861986CD
:1050F00080918E0490918F049A838983FC82EB8245
:10510000809192048D83DF82B6CF0E94EE130E94BD
:1051100083158816990608F058C0511409F44FCD2C
:10512000611409F44EC090918F04F80181819813A5
:1051300030C090918E04808198132BC08091900490
:1051400090919104E81AF90A60E08EE894E00E94D8
:10515000EE138091BB049091BC04E816F90608F0A8
:1051600063CF8091940480FD5FCF803108F45CCFE1
:10517000D80116968C931697982F907F903F09F43C
:1051800050CF982F907F905F8F70892B16968C93BD
:1051900048CFC8010E94C013811571F0609142048C
:1051A00070914304C80170DC811509F4FFCC89E0DB
:1051B000EEE8F4E0DF0186CF809194048160809373
:1051C0009404C8010E947B18FACC89E0F501119281
:1051D0008A95E9F782CDA1E2B0E0E1EFF8E20C9424
:1051E00069334C8F5D8F6E8F7F8F082F88A3192FA7
:1051F00099A3F82EE92E811509F4A3C040E0692F88
:105200008C8D9D8D0E94D2139C01111549F0109236
:10521000C3049093C2048093C10410923E040AC058
:105220008091C1049091C2048217930719F481E020
:105230008093C304198E1A8E1B8E86E0FE017C9625
:10524000DE01539601900D928A95E1F78091C0049A
:1052500082FF21C08091990490919A04892BD9F002
:105260000E94CB092091400430914104821B930B92
:105270002091990430919A048217930738F0809115
:105280003F0482FD03C082E00E9450050E94D709BE
:1052900081110E948105F11461F00F8B188F61E07C
:1052A000CE0143960E94EE1361E0CE0143960E9428
:1052B000EE130F8B188F89E0FE017396DE011A96AC
:1052C00001900D928A95E1F7CE010A9629DC8111B1
:1052D00010C0209144043091450489E0FE013A96C3
:1052E000DE01119601900D928A95E1F78E8581116C
:1052F0002CC019E08091450490914404891741F035
:10530000189FC00111248A5B9B4F0ADC811144C0A5
:105310008E85811112C08091140181110EC08C857F
:105320009D852091420430914304821B930B8F3F53
:105330009F4318F081E080931401A196E6E00C945D
:105340008533911509F476CF68CF822F90E00196CE
:10535000877099273817190671F40E94540E10921D
:1053600044041092450489E0EEE8F4E0DF011D9268
:105370008A95E9F7BECF99E0929FD0011124AA5BEC
:10538000BB4FFE01319601900D929A95E1F7809303
:1053900044040E944605ADCF8091450490E00196FB
:1053A0008770992780934504A5CFA6E0B0E0EBED88
:1053B000F9E20C946B330E94CB098C01809154026A
:1053C000909155028017910771F019821A820E94FC
:1053D000CB09BC0149815A8180E090E0FCDE10934A
:1053E0005502009354022696E4E00C948733A6E01D
:1053F000B0E0EDEFF9E20C946D339093510280939D
:105400005002811520E2920730F40E94D70D2696B3
:10541000E2E00C94893380EF89838A830E94CB0970
:105420008160BC0149815A8181E091E0D4DEEFCFF7
:10543000A6E0B0E0EEE1FAE20C946D3390935102F5
:1054400080935002811520E2920730F40E941E0ED4
:105450002696E2E00C94893380EF89838A830E9448
:10546000CB098160BC0149815A8181E090E0B3DEC3
:10547000EFCFCF93DF93D82FC92FB9DF8091B50439
:105480009091B6040E94350C8D2F9C2FD1DFDF91B7
:10549000CF9108950F931F93CF93DF938C01862FA5
:1054A0006EE073E00E946E15892B91F4C0910E039B
:1054B000D0910F03209761F0F8018281833039F495
:1054C000CE01D7DFCE01D5DFCE01D3DF01C0E0F7BB
:1054D000DF91CF911F910F9108950F931F93CF9359
:1054E000DF938C01EB016EE073E08C2F0E946E1550
:1054F000892B09F057C0FE01FF27D80112968C9125
:105500001297E95EFD4F8130A9F415968C9182FDCA
:105510004EC080FF4CC082E0808380911003909148
:1055200011030097B9F480910E0390910F03009737
:10553000C9F110C08230A1F515968C9182FD26C06C
:1055400080FD0AC083E08083809112039091130351
:105550000097F1F04CDF26C084E080838091140333
:10556000909115030097B1F780910E0390910F036E
:10557000009701F17EDF8091100390911103009755
:1055800049F780910E0390910F03E4CF85E080836B
:1055900080910E0390910F03009721F06ADFF1CF05
:1055A00086E08083DF91CF911F910F91089581E074
:1055B0008083B9CF8091100390911103B8CF0F93DE
:1055C0001F93CF93DF938C01EB016EE073E08C2F80
:1055D0000E946E15892BA1F48091B5049091B604B8
:1055E0000E94350CDD27C95EDD4F8881F8011282EB
:1055F00018828330E9F048F4813059F0823081F02C
:10560000DF91CF911F910F9108958430B1F08530D3
:10561000B9F780910E0390910F03009789F306C0AC
:105620008091100390911103009799F301DFE8CF67
:105630008091120390911303F7CF809114039091FE
:105640001503009799F720910E0330910F03809175
:1056500010039091110321153105F9F2009731F7EC
:10566000C901E4CFCDB7DEB7AC970FB6F894DEBF73
:105670000FBECDBF85B7806885BF85B7806885BF01
:1056800084B7877F84BF0FB6F894A8958091600097
:10569000886180936000109260000FBE80E890E007
:1056A0000FB6F89480936100909361000FBE81E083
:1056B000809311018BE797E09093AD018093AC014B
:1056C0000E94A3070E94AF140E942E150E94E612AA
:1056D0000E945F0B0E94BC0B8091E200846080936B
:1056E000E200789480914F02811599F08091E90051
:1056F0001091EC008F70179511271795182B1092A9
:10570000E9008091E80083FD0E94C00E1F70109395
:10571000E90082E084BD93E095BD9AEF97BD809348
:105720006E000E940914811102C00E94AD170DE2A3
:1057300011E0D8018D918D018F3F11F00E947D07FE
:10574000B1E002331B07A9F702E311E0A0E4EA2E5F
:10575000A1E0FA2EF80181918F018F3F11F00E9494
:105760007D07E016F106B1F78AE0E3E4F2E0DF013D
:10577000282F1D922A95E9F7EFE1F2E0DF011D9253
:105780008A95E9F780E090E00E94D233833E9E4FF5
:1057900021F40E940914811129C063EE7EEF80E09C
:1057A00090E00E94003460E082E090E00E94E633E6
:1057B00081E08093390461E083E090E00E94E63369
:1057C00060E074E184E090E00E9400340E94AD1734
:1057D00040E050E0BA018FE090E00E94F83340E0F2
:1057E00050E0BA0183E190E00E94F83382E090E05B
:1057F000D1D780932B0284E090E0D4D79093C0045B
:105800008093BF040E94C316EFEFF6E721E0E1505A
:10581000F0402040E1F700C000000E94C3168091D4
:10582000430280FF07C06FEF7FEF80E090E0E8D792
:105830000E94430C83E090E0ADD70E942E0480E0EC
:1058400091E0909377028093760280914F028530A9
:1058500049F480914F02853009F45CC00E94540ED7
:105860000E9409090E94C316FCE2AF2EF2E0BF2E8F
:1058700003E412E0D801F501219131918D919D91C0
:1058800046E352E04E175F0709F47AC0281739073C
:1058900099F3E3E48E2EE2E09E2E512CD401ED909C
:1058A000FD904D01F501619071905F016E147F04D0
:1058B00051F16E247F24412CCC24C394D12CC301FC
:1058C0008C219D21892BB1F049825A820E94CB09FB
:1058D0009C838B83F1E0FD8391E097012C213D2196
:1058E000232B09F490E09E8349815A816B817C814E
:1058F0008D8171DC4394CC0CDD1C2EE04212DFCF95
:10590000F501F292E292539435E05312C7CF0E9410
:10591000680A3BC080914F02843021F11092290225
:1059200048E150E080E40FB6F894A89540936000F9
:105930000FBE8093600083B7817F846083BF83B78D
:10594000816083BF7894889583B78E7F83BF0FB6BD
:10595000F894A8958091600088618093600010920F
:1059600060000FBE0E94C316E3E4F2E081919191C2
:10597000892B09F0BCC492E0ED34F907B9F769CF7F
:105980002817390709F085CF10DDE0909903F090D2
:105990009A03E114F10491F180903A0290903B0255
:1059A000A0903C02B0903D020E94680A68197909F3
:1059B0008A099B098090360290903702A0903802A5
:1059C000B0903902681579058A059B05B8F0C701C2
:1059D0000E94D70D10929A031092990310923A02E6
:1059E00010923B0210923C0210923D02109236023D
:1059F000109237021092380210923902C09021049E
:105A0000D0902204C114D10439F1A0902304B090A5
:105A100024040E94CB097C01EA18FB08C6010E94FD
:105A200083158E159F05C0F4209121043091220426
:105A3000C9019927287F3327232B09F080C054E020
:105A4000880F991F5A95E1F78F559C4FDC011596E9
:105A50002C9122FF0E9448128091B20480FF1CC04A
:105A60008091130182FF18C00E94CB09BC01809174
:105A70002504909126049B01281B390B80910C0171
:105A800090910D012817390738F041E080912704E3
:105A9000909128040E94A41180911803811569F047
:105AA0000E94CB092091190330911A03821B930B9A
:105AB0008F3F9F4710F40E94720D0E940909909138
:105AC0003E02891721F080933E020E94680A80916D
:105AD0004F02843009F0B9CE83E08093E9008091D1
:105AE000E80082FFB2CE8091E80090E085FF05C01B
:105AF0000E942E0B811531F191E08091E8008B77A7
:105B00008093E800911509F4A0CEE0905202F09045
:105B10005302E981E114F10499F1EE3F09F051C01B
:105B20008A81833020F08550833008F04AC0EA81B2
:105B3000EE3008F046C0F0E0E25DFB4CA1C580E02D
:105B400090E084CF40E2C42ED12CFE0131967F013B
:105B50008091E80085FD0AC08091E8008B778093F2
:105B6000E8000E942E0B811599F3C6CF8091F100B9
:105B7000D7018D937D01B1E0CB1AD10849F7BCCF95
:105B8000E43148F4E11549F0E150E33130F4F0E05C
:105B9000E45CFB4C75C5EE3F51F28FEFD4C31A8223
:105BA00089E08B830EC08A81823081F08330B1F02E
:105BB000813099F70E94680A79D56B837C838D8345
:105BC0009E83CE0101960E947E0B3FCE88E290E03C
:105BD000E1D51B821C821D828E83F3CF80914D0202
:105BE00090914E02892B69F3FE013196D8018C9178
:105BF00011969C910E5F1F4F928383833296B2E081
:105C00000D341B0799F7DDCF8A81823031F66B8125
:105C10007C818D819E814AD588E290E0D7D5D1CF15
:105C20004C816B818A810E943F139827892798278E
:105C30009E838D83C6CF2D813E8132272327322735
:105C40004C816B818A810E94DF0CBBCF0E942214A1
:105C5000B8CF80E18A83B5CF1A828FEAA2CF8C8138
:105C60008D3108F0AECF8A809B80982489249824B7
:105C7000A12CB12C8E010F5F1F4F7801E80EF11C93
:105C8000E016F10609F49DCF80E0EFEA8E1691044C
:105C9000A104B10420F4C4018F5A9C4F7BD5D801D4
:105CA00014968C930F5F1F4FBFEF8B1A9B0AAB0AA2
:105CB000BB0AE6CF80914D0290914E02892B09F4E8
:105CC00080CF8C818D3108F07CCF882E912CA12C37
:105CD000B12CCA80DB80DC24CD24DC24E12CF12C27
:105CE0008E010F5F1F4F412C512C32014814590473
:105CF0006A047B0408F065CFEFEACE16D104E10414
:105D0000F10438F4D80114966C91C6018F5A9C4F57
:105D10005DD5BFEF4B1A5B0A6B0A7B0AEFEFCE1A19
:105D2000DE0AEE0AFE0A0F5F1F4FE0CF0E947317D4
:105D300048CF84E08FCF8C818D3108F042CF882E00
:105D4000912CA12CB12CCA80DB80DC24CD24DC2456
:105D5000E12CF12C412C512C32018E010B5F1F4F95
:105D6000481459046A047B0408F02BCF80E0F0E368
:105D7000CF16F2E0DF06E104F10418F4C6018996BB
:105D800009D5D8018D938D01BFEF4B1A5B0A6B0AC1
:105D90007B0AEFEFCE1ADE0AEE0AFE0AE1CF2C8173
:105DA000022F10E02D3108F00CCF8A819B819827BB
:105DB000892798272C01612C712C8033F2E09F07F2
:105DC00008F0FFCE822E912CA12CB12C40E352E0A2
:105DD00060E070E0441955096609770942175105DA
:105DE0006105710508F4EDCE20914D0230914E020F
:105DF000232B09F03EC01C0129E2220E311C80FB3E
:105E0000EE24FF24E0F880FF0BC08896C3D49D8168
:105E100089279827892781159C4711F48FEF8D8357
:105E2000D501C401840D951DA61DB71D80FF19C0A5
:105E3000680141E0C41AD108CE0105968C0D9D1D64
:105E40009CA78BA7C101800F911FA4D4ABA5BCA5B3
:105E50009C9181159C4721F48FEFEBA5FCA58083D5
:105E60008601FE013196EE0DFF1D2FEFE016F106C3
:105E700038F08E010F5F1F4FC12CD12C760125C049
:105E80009481858181159C4711F42483258342E008
:105E9000E40EF11C3296EACF50E3451652E0550667
:105EA0006104710430F4D80114966C91C201899692
:105EB0008DD4BFEFCB1ADB0AEB0AFB0AEFEF4E1AC9
:105EC0005E0A6E0A7E0A0F5F1F4FC814D904EA04E7
:105ED000FB0410F376CE80914D0290914E02892BF7
:105EE00009F46FCECE0101960E947E0BFFEF21EEEA
:105EF00034E0F15020403040E1F700C0000098CC81
:105F000088E0E5E1F1E0DE01919601900D928A953D
:105F1000E1F7FE0132968FE1DF011D928A95E9F7E4
:105F200086E0898388E07F96DE01159601900D92C8
:105F30008A95E1F746CE80EE898381E08A831B82D1
:105F40001C823FCE8B819C81092E000CAA0BBB0BBF
:105F500035E0880F991FAA1FBB1F3A95D1F7AC01F6
:105F6000BD01405E5F4F6F4F7F4F481759076A076B
:105F70007B0708F426CE803EE1E09E07A105B1052F
:105F800008F01FCE413EF1E05F076105710520F08A
:105F900040EE51E060E070E0481B590BBC016E53CD
:105FA0007B4FCE010196C0D30CCE4AE150E06FEF9B
:105FB00070E0CE010796D7D380914D028983EA82A3
:105FC0001B821C8284E08D838DE006CE81E090E010
:105FD000909353028093520282E390E090934202A6
:105FE000809341020E94CB099093400280933F022C
:105FF000E8CDE114F10481F1D0904302C0904C024D
:1060000000913F02109140020E94CB09801B910B2E
:106010008536910540F1C5FE26C0D0FE24C00E9401
:10602000CB099093400280933F028091410290916E
:10603000420201979093420280934102892B61F4BE
:10604000109253021092520281E090E090934E021F
:1060500080934D02E12CF12C80914D028983EA82DC
:10606000809141029ECD82E390E090934202809322
:106070004102F2CF10924E0210924D02A2CD0B813E
:106080001C8140E250E06FEF70E0CE0101966BD3CF
:1060900026EF33E042E050E080E090E0F9016591C6
:1060A00075910617170740F4DE0111968A0F9B1FA2
:1060B000FC0171836083CA01F4E0263B3F0709F4C9
:1060C00080CDAC014E5F5F4F245F3F4F41325105A1
:1060D00028F377CD2B813C8186EF93E0FC0145913D
:1060E00055914217530709F41FC10C9644E0823CB6
:1060F0009407A1F752CD8B819C8106EF13E0F80144
:10610000259135918217930709F41FC1045F1F4F32
:10611000F4E0023C1F0799F7EE24EA94FE2C30C10C
:106120000E940C134ECDEB81E93008F04ACDF0E02F
:10613000E15BFB4CA5C2FE0132968EE1DF011D92B0
:106140008A95E9F788E089838B838C8383E088A331
:1061500038CD8C819AE0F92E8E010F5D1F4FF8012A
:106160002F2D11922A95E9F7B8010E946E158983A7
:10617000F801DE01129601900D92FA94E1F721CD1B
:106180001C818AE0FE013596DE01919601900D9208
:106190008A95E1F789A19AA10E9496079AA389A3FB
:1061A0008BA19CA10E9496079CA38BA38DA19EA16D
:1061B0000E9496079EA38DA38FA198A50E94960783
:1061C00098A78FA38FEF183060F43AE0139FB001C7
:1061D00011246F577D4F4AE050E0CE01819614D3D1
:1061E00080E089830E94A307ECCC2C816AE0CE0179
:1061F0008196DC01E62F1D92EA95E9F7283080F4BC
:10620000629FB00111246F527D4F4AE050E0B2D23C
:1062100080E089838AE0FE01B196DE01129686CE87
:106220008FEFF7CF1C818AE0FE013596DE01919653
:1062300001900D928A95E1F78BA19CA10E9496078F
:106240009CA38BA38FEF183060F4FAE01F9FB0017E
:1062500011246F527D4F4AE050E0CE018196D4D296
:1062600080E089830E94AF14ACCC2C8166E0CE0123
:106270008196DC01E62F1D92EA95E9F7283060F45B
:10628000629FB00111246F5D7C4F46E050E072D2F6
:1062900080E0898386E0BFCF8FEFFBCF1C8186E053
:1062A000FE013596DE01919601900D928A95E1F7F7
:1062B00089A19AA10E9496079AA389A38BA19CA168
:1062C0000E9496079CA38BA38FEF183060F4F6E032
:1062D0001F9FB00111246F5D7C4F46E050E0CE015E
:1062E000819692D280E089830E942E156ACC80919B
:1062F0002A02811509F4ADCAA0E1A9BDB2E1B9BD78
:1063000009B400FEFDCF8091D8008F7D8093D80026
:106310008091E00082608093E0008091E00081FD48
:10632000FCCF0E94540E95CAFC01369625913591FA
:106330002115310509F431CC4FE150E0BE016E5F0B
:106340007F4FF901099589833CCCF8013896259156
:1063500035912115310509F4DFCE4CE150E0BE0145
:106360006B5F7F4FC801F90109957C01892B41F4CE
:10637000F8013A9685919591009711F0FC010995E5
:10638000E9821FCC1F921FB61F9211248F939F93F7
:10639000AF93BF9380912902811113C08091EE01C8
:1063A0009091EF01A091F001B091F1014196A11DF2
:1063B000B11D8093EE019093EF01A093F001B09393
:1063C000F101BF91AF919F918F911F901FBE1F90C0
:1063D000189578941F921FB61F9211248F939F9344
:1063E000AF93BF938091EE019091EF01A091F001E6
:1063F000B091F1010196A11DB11D8093EE01909322
:10640000EF01A093F001B093F101BF91AF919F9183
:106410008F911F901FBE1F9018951F920F920FB65D
:106420000F9211242F933F934F935F936F937F931A
:106430008F939F93AF93BF93EF93FF938091E1006E
:1064400082FF09C08091E20082FF05C08091E100D7
:106450008B7F8093E1008091DA0080FF24C08091DF
:10646000D80080FF20C08091DA008E7F8093DA0010
:106470008091D90080FFA9C080E189BD82E189BDFA
:1064800009B400FEFDCF81E080934F028091DD01D1
:10649000811109C00E945F0B0E94BC0B8091E20039
:1064A00084608093E2008091E10080FF1AC08091B7
:1064B000E20080FF16C08091E2008E7F8093E200B0
:1064C0008091E20080618093E2008091D800806238
:1064D0008093D80019BC85E080934F0283E08093BD
:1064E00011018091E10084FF2FC08091E20084FFC0
:1064F0002BC080E189BD82E189BD09B400FEFDCFDA
:106500008091D8008F7D8093D8008091E1008F7EAC
:106510008093E1008091E2008F7E8093E200809181
:10652000E20081608093E2008091DC01811509F432
:1065300052C084E080934F0280914F02843009F072
:1065400052C082E0809311018091E10083FF2CC052
:106550008091E20083FF28C08091E100877F8093D3
:10656000E10082E080934F021092DC018091E10013
:106570008E7F8093E1008091E2008E7F8093E20025
:106580008091E20080618093E20042E060E080E080
:106590000E948C0B8091F00088608093F00081E075
:1065A0008093110180931001FF91EF91BF91AF9102
:1065B0009F918F917F916F915F914F913F912F911B
:1065C0000F900FBE0F901F90189519BC10924F029C
:1065D0001092DD0168CF8091E30087FF02C083E065
:1065E000A9CF81E0A7CF81E0ADCF1F920F920FB668
:1065F0000F921124EF92FF920F931F932F933F93CB
:106600004F935F936F937F938F939F93AF93BF93BA
:10661000CF93EF93FF9309EE10E0F8018081C091D2
:10662000EC008F70C795CC27C795C82B108280EFE0
:10663000E82EF12CF7018081877F808378940E9477
:10664000C00EF8011082F701808188608083CF70CE
:10665000F801C083FF91EF91CF91BF91AF919F91CE
:106660008F917F916F915F914F913F912F911F91EA
:106670000F91FF90EF900F900FBE0F901F90189505
:10668000EE0FFF1F0590F491E02D0994082E817004
:1066900006940694811D0694811D0694811D06941E
:1066A000811D0694811D0694801D089569279627F3
:1066B000692778278727782708952F923F924F924E
:1066C0005F926F927F928F929F92AF92BF92CF9282
:1066D000DF92EF92FF920F931F93CF93DF93CDB78B
:1066E000DEB7CA1BDB0B0FB6F894DEBF0FBECDBF03
:1066F00009942A88398848885F846E847D848C84D4
:106700009B84AA84B984C884DF80EE80FD800C81DC
:106710001B81AA81B981CE0FD11D0FB6F894DEBFBF
:106720000FBECDBFED010895FB01DC0102C0059055
:106730000D9241505040D8F70895FB01DC0104C090
:106740008D910190801921F441505040C8F7881B69
:10675000990B0895FB01DC0102C001900D9241509C
:106760005040D8F70895DC0101C06D93415050406E
:10677000E0F70895DC01CB01FC01F999FECF06C0DA
:10678000F2BDE1BDF89A319600B40D9241505040EF
:10679000B8F70895F999FECF92BD81BDF89A99276F
:1067A00080B50895A8E1B0E042E050E0E5CFDC011B
:1067B000A40FB51F4150504040F0CB01840F951FEE
:1067C0002E9105D041505040D8F70895262FF999C1
:1067D000FECF92BD81BDF89A019700B4021639F040
:1067E0001FBA20BD0FB6F894FA9AF99A0FBE089511
:1067F0000396272FECDFEADF252FE9DF242FE7CFF1
:106800000196272FE4DFE2CFDC01CB0102C02D91FE
:1068100005D041505040D8F70895262FF999FECF62
:106820001FBA92BD81BD20BD0FB6F894FA9AF99AAD
:106830000FBE01960895F894FFCF9D0FC30FC90FA7
:10684000C30FC90F1B103C10C90F42114F119020EC
:10685000962082208A209C20A220A820802F9B2F77
:10686000A22FE12DE12DD52FE62FF92F3A303F3021
:106870006A307B3090309330CF2DD32D042E102EE4
:106880001B2E262ECD2DCD2DCD2DCD2D6B2F292E92
:106890002C2E2F2E5A2E962E992E9B2ECF2E9B309D
:1068A000A930C030E12DE12DF530123135314E31B6
:1068B000C809A90CBF0CB50AC40CA00CAF0000009D
:1068C00001000101011AF059B1D95B753000442271
:1068D0006D3B011901AC0041025A027A029491F712
:1068E000F6F537F0F1F4676636353497969593925E
:1068F000E200E900EA00B500B600B700CD00830170
:10690000CC008A0192019401210223022402250273
:10691000260227022A02B300B4006F0070009F0114
:10692000CB019F02A002E200E900EA00B500B60038
:10693000B700CD008301CC008A01920194012102AD
:10694000230224022502260227022A02B300B400F1
:0C6950006F0070009F01CB019F02A002AD
:00000001FF
